:020000040000FA
:040800002AEF08F0E3
:1008100003B213EF05F0F2B431EF05F09EB039EFFB
:1008200005F09EB241EF05F0F2A81AEF04F0F2B223
:1008300025EF04F0F2A620EF04F0F2B022EF04F06E
:10084000D9EF07F0F296F290FF00CD90F2929EA0C1
:100850002FEF04F00101533F2FEF04F0542BAEC1F2
:10086000B2F1AFC1B3F1B0C1B4F1B1C1B5F1AAC138
:10087000AEF1ABC1AFF1ACC1B0F1ADC1B1F1A6C148
:10088000AAF1A7C1ABF1A8C1ACF1A9C1ADF1A2C158
:10089000A6F1A3C1A7F1A4C1A8F1A5C1A9F19EC168
:1008A000A2F19FC1A3F1A0C1A4F1A1C1A5F19AC178
:1008B0009EF19BC19FF19CC1A0F19DC1A1F196C188
:1008C0009AF197C19BF198C19CF199C19DF1CECF4E
:1008D00096F1CFCF97F153C198F154C199F1CF6AF6
:1008E000CE6A0101536B546B9E90CD800FBC0F8E6E
:1008F0000FBA7EEF04F00F8AD9EF07F00F8C0FBE0E
:10090000BAEF04F096C19AF197C19BF198C19CF19E
:1009100099C19DF19AC19EF19BC19FF19CC1A0F12B
:100920009DC1A1F19EC1A2F19FC1A3F1A0C1A4F1FB
:10093000A1C1A5F1A2C1A6F1A3C1A7F1A4C1A8F1CB
:10094000A5C1A9F1A6C1AAF1A7C1ABF1A8C1ACF19B
:10095000A9C1ADF1AAC1AEF1ABC1AFF1ACC1B0F16B
:10096000ADC1B1F1AEC1B2F1AFC1B3F1B0C1B4F13B
:10097000B1C1B5F101015E6B5F6B606B616B96514C
:100980005E2797515F2398516023995161239A51B3
:100990005E279B515F239C5160239D5161239E5193
:1009A0005E279F515F23A0516023A1516123A25173
:1009B0005E27A3515F23A4516023A5516123A65153
:1009C0005E27A7515F23A8516023A9516123AA5133
:1009D0005E27AB515F23AC516023AD516123AE5113
:1009E0005E27AF515F23B0516023B1516123B251F3
:1009F0005E27B3515F23B4516023B5516123D89072
:100A00000101613360335F335E33D890010161339C
:100A100060335F335E33D8900101613360335F33FD
:100A20005E33D9EF07F00392ABB2AB98AB8803010A
:100A300003EE00F080517F0BE92604C0EFFF802B0E
:100A40008151805D700BD8A48B8200008051815D44
:100A5000700BD8A48B9281518019D8B40790D9EF2C
:100A600007F0F2940101453FD9EF07F0462BD9EF8B
:100A700007F09E900101533FD9EF07F0542BD9EFB7
:100A800007F09E92040062A146EF05F007B498EFCC
:100A900005F007B098EF05F01EC620F61FC621F638
:100AA0001CC61EF61DC61FF61AC61CF61BC61DF672
:100AB00006C608F607C609F604C606F605C607F612
:100AC00002C604F603C605F626C628F627C629F68A
:100AD00024C626F625C627F622C624F623C625F602
:100AE0000EC610F60FC611F60CC60EF60DC60FF6A2
:100AF0000AC60CF60BC60DF62EC630F62FC631F61A
:100B00002CC62EF62DC62FF62AC62CF62BC62DF691
:100B100016C618F617C619F614C616F615C617F631
:100B200012C614F613C615F696EC2AF02EEC2AF02F
:100B3000077C07ACB3EF05F0C274C2B4ADEF05F0AB
:100B4000C3CFB3F5C4CFB4F50501D890B433B333F4
:100B5000D890B433B333B4EF05F0C3CF55F1C4CF5D
:100B600056F1B4EF05F0C28207B421EF06F047C199
:100B70004BF148C14CF149C14DF14AC14EF15EC142
:100B800062F15FC163F160C164F161C165F196C159
:100B9000B6F197C1B7F198C1B8F199C1B9F19AC14D
:100BA000BAF19BC1BBF19CC1BCF19DC1BDF19EC11D
:100BB000BEF19FC1BFF1A0C1C0F1A1C1C1F1A2C1ED
:100BC000C2F1A3C1C3F1A4C1C4F1A5C1C5F1A6C1BD
:100BD000C6F1A7C1C7F1A8C1C8F1A9C1C9F1AAC18D
:100BE000CAF1ABC1CBF1ACC1CCF1ADC1CDF1AEC15D
:100BF000CEF1AFC1CFF1B0C1D0F1B1C1D1F1B2C12D
:100C0000D2F1B3C1D3F1B4C1D4F1B5C1D5F1B3C5FB
:100C1000B5F5B4C5B6F5B5C5B7F5B6C5B8F50101B6
:100C200055515B2756515C23E86A5D230E2E21EF58
:100C300006F05CC157F15DC158F15B6B5C6B5D6B9D
:100C4000078E0201002FD9EF07F03C0E006F05015F
:100C50002F51000AD8B4D8EF06F005012F51010A30
:100C6000D8B462EF06F005012F51020AD8B4A3EF01
:100C700006F005012F51030AD8B4A3EF06F00501D1
:100C80002F51040AD8B4A3EF06F005012F51050A2D
:100C9000D8B4A3EF06F005012F51060AD8B4A3EF8C
:100CA00006F005012F51070AD8B4A3EF06F005019D
:100CB0002F51320AD8B460EF06F02F6BD8EF06F050
:100CC000D8EF06F0050153676DEF06F054676DEF3E
:100CD00006F055676DEF06F0566771EF06F0D8EF36
:100CE00006F057C500F158C501F159C502F15AC5C2
:100CF00003F10101010E046F000E056F000E066F77
:100D0000000E076F9FEC28F000C157F501C158F5A0
:100D100002C159F503C15AF5006796EF06F0016765
:100D200096EF06F0026796EF06F00367D8EF06F03D
:100D300053C557F554C558F555C559F556C55AF517
:100D40000F88D8EF06F005013067A9EF06F0D8EF5D
:100D500006F00FBEBEEF06F010A0C3EF06F00101D3
:100D60004767BAEF06F04867BAEF06F04967BAEF8F
:100D700006F04A67BEEF06F0C3EF06F007AEC3EF1A
:100D800006F0D5EF06F00501312FD8EF06F03C0E46
:100D9000316F302FD8EF06F00101000E626FE00EC8
:100DA000636FA50E646F010E656F0501306B0F88D0
:100DB0000501626B33B7DEEF06F062810CC100F112
:100DC0000DC101F10EC102F10FC103F110C104F117
:100DD00011C105F112C106F113C107F114C108F1E7
:100DE00015C109F116C10AF117C10BF135C134F172
:100DF00000C10CF101C10DF102C10EF103C10FF1EF
:100E000004C110F105C111F106C112F107C113F1BE
:100E100008C114F109C115F10AC116F10BC117F18E
:100E200034C135F101018A671DEF07F08B671DEFB3
:100E300007F08C671DEF07F08D6721EF07F051EF8A
:100E400007F08EC100F18FC101F190C102F191C193
:100E500003F10101010E046F000E056F000E066F15
:100E6000000E076F9FEC28F000C18EF101C18FF1D9
:100E700002C190F103C191F1006746EF07F00167ED
:100E800046EF07F0026746EF07F0036751EF07F000
:100E90008AC18EF18BC18FF18CC190F18DC191F11E
:100EA0000F80D57ED5BE69D0D6CF47F1D7CF48F1D8
:100EB00045C149F1E86AE8CF4AF1109047C100F115
:100EC00048C101F149C102F14AC103F101010A0E11
:100ED000046F000E056F000E066F000E076F9FEC8B
:100EE00028F003AF1080010154A783EF07F00F9A99
:100EF0000F9C0F9E0101000E5E6F600E5F6F3D0E36
:100F0000606F080E616F010147BF93EF07F04867FC
:100F100093EF07F0496793EF07F04A6793EF07F005
:100F2000F288B8EF07F0F2985E6B5F6B606B616BF5
:100F3000966B976B986B996B9A6B9B6B9C6B9D6B8D
:100F40009E6B9F6BA06BA16BA26BA36BA46BA56B3D
:100F5000A66BA76BA86BA96BAA6BAB6BAC6BAD6BED
:100F6000AE6BAF6BB06BB16BB26BB36BB46BB56B9D
:100F7000D76AD66A0101456B466B0CC100F10DC101
:100F800001F10EC102F10FC103F110C104F111C151
:100F900005F112C106F113C107F114C108F115C121
:100FA00009F116C10AF117C10BF135C134F1D9EFBE
:100FB00007F002C0E0FF005001C0D8FF1000A6B249
:100FC000DFEF07F00CC0A9FF0BC0A8FFA69EA69CF0
:100FD000A684F29E550EA76EAA0EA76EA682F28E6A
:100FE000A694A6B2F1EF07F00C2A1200A96EA69EF5
:100FF000A69CA680A8500C2A120004012C0E826F19
:101000001AEC0BF09AEC29F00C50F6EC07F0E8CF54
:1010100000F10C50F6EC07F0E8CF01F101AF16EF4C
:1010200008F00101FF0E026FFF0E036F3DEC29F087
:10103000296722EF08F00401200E826F1AEC0BF0F2
:1010400027EF08F004012D0E826F1AEC0BF067EC0D
:1010500027F01200076A0F6A106A0F010D0EC16EA9
:10106000860EC06E030EC26E0F01680E896E130EDF
:10107000926E080E8A6E8A6AF30E936E8B6A900ED9
:10108000946EF18EF19E0E6A01015B6B5C6B5D6B81
:10109000576B586BF29A0101476B486B496B4A6B6F
:1010A0004B6B4C6B4D6B4E6B4F6B506B516B526B74
:1010B000456B466BD76AD66A0F01280ED56EF28A49
:1010C0009D90B00ECD6E01015E6B5F6B606B616BCE
:1010D000626B636B646B656B666B676B686B696B8C
:1010E000536B546BCF6ACE6A0F9A0F9C0F9E9D80F4
:1010F000760ECA6E9D8202013C0E006FCC6A160EFF
:10110000F6EC07F0E8CF00F1170EF6EC07F0E8CFA9
:1011100001F1180EF6EC07F0E8CF02F1190EF6EC2B
:1011200007F0E8CF03F1010103AFB1EF08F09AEC4B
:1011300029F0160E0C6E00C10BF0DFEC07F0170E55
:101140000C6E01C10BF0DFEC07F0180E0C6E02C143
:101150000BF0DFEC07F0190E0C6E03C10BF0DFECA7
:1011600007F000C18AF101C18BF102C18CF103C10A
:101170008DF100C18EF101C18FF102C190F103C167
:1011800091F11A0EF6EC07F0E8CF00F11B0EF6EC29
:1011900007F0E8CF01F11C0EF6EC07F0E8CF02F102
:1011A0001D0EF6EC07F0E8CF03F1010103AF07EFE6
:1011B00009F09AEC29F01A0E0C6E00C10BF0DFEC6E
:1011C00007F01B0E0C6E01C10BF0DFEC07F01C0EDC
:1011D0000C6E02C10BF0DFEC07F01D0E0C6E03C1AC
:1011E0000BF0DFEC07F01A0EF6EC07F0E8CF00F199
:1011F0001B0EF6EC07F0E8CF01F11C0EF6EC07F041
:10120000E8CF02F11D0EF6EC07F0E8CF03F100C1C4
:1012100092F101C193F102C194F103C195F1240E41
:10122000AC6E900EAB6E240EAC6E080EB86E000E57
:10123000B06E1F0EAF6E0401806B816B0F01900EBC
:10124000AB6E0F019D8A0301806B816BC26B8B9229
:1012500029EC30F029EC30F0880EF6EC07F0E8CFFE
:1012600000F1890EF6EC07F0E8CF01F1010101AFC2
:1012700052EF09F09AEC29F0880E0C6E00C10BF0C9
:10128000DFEC07F0890E0C6E01C10BF0DFEC07F00C
:10129000880EF6EC07F0E8CF00F1890EF6EC07F0C7
:1012A000E8CF01F100C140F601C141F602C142F6AA
:1012B00003C143F681EC33F00AEC2EF0200EF6EC7D
:1012C00007F0E8CF2FF505012F51FF0AD8A470EFE2
:1012D00009F02F6B200E0C6E2FC50BF0DFEC07F022
:1012E0000501010E306F3C0E316F250EF6EC07F054
:1012F000E8CF00F1260EF6EC07F0E8CF01F1270E5B
:10130000F6EC07F0E8CF02F1280EF6EC07F0E8CF94
:1013100003F1010103AFA7EF09F09AEC29F0250EC4
:101320000C6E00C10BF0DFEC07F0260E0C6E01C155
:101330000BF0DFEC07F0270E0C6E02C10BF0DFECB8
:1013400007F0280E0C6E03C10BF0DFEC07F000C1B4
:1013500053F501C154F502C155F503C156F500C15D
:1013600057F501C158F502C159F503C15AF5290EC7
:10137000F6EC07F0E8CF5BF505015C515B5DD8A0AA
:101380005BC55CF505012F51020A0EE181B8D4EF6F
:1013900009F005015C2FD1EF09F05BC55CF5D4EFD6
:1013A00009F081BAC0EF33F0210EF6EC07F0E8CF78
:1013B00000F1220EF6EC07F0E8CF01F1230EF6EC77
:1013C00007F0E8CF02F1240EF6EC07F0E8CF03F1C6
:1013D000010103AF1AEF0AF09AEC29F0210E0C6E0E
:1013E00000C10BF0DFEC07F0220E0C6E01C10BF018
:1013F000DFEC07F0230E0C6E02C10BF0DFEC07F000
:10140000240E0C6E03C10BF0DFEC07F0210EF6EC9E
:1014100007F0E8CF00F1220EF6EC07F0E8CF01F17B
:10142000230EF6EC07F0E8CF02F1240EF6EC07F0FD
:10143000E8CF03F100C15DF501C15EF502C15FF5C2
:1014400003C160F541EC2DF003EC2CF053EC2BF0D4
:1014500005012F51030A12E005012F51040A1DE076
:1014600005012F51050A24E005012F51060A32E03B
:1014700005012F51070A38E07DEF0AF0ACC500F1F5
:1014800001010F0E001701010051000A36E00101B1
:101490000051050A32E07AEF0AF0ACC500F1010113
:1014A0000F0E001701010051000A27E07AEF0AF041
:1014B0000501AC51000A21E00501AC51150A1DE0FF
:1014C0000501AC51300A19E00501AC51450A15E09F
:1014D0007AEF0AF00501AC51000A0FE00501AC51AA
:1014E000300A0BE07AEF0AF00501AC51000A05E082
:1014F0007AEF0AF081BAC0EF33F0FEEC2AF00790E1
:101500000001F28EF28C07B0FBEF24F00FB0DCEF9D
:101510001FF00FB8A0EF19F00301805181197F0B64
:10152000D8B4FBEF24F013EE00F081517F0BE126DD
:10153000812BE7CFE8FFE00BD8B4FBEF24F023EEDC
:1015400082F0C2513F0BD926E7CFDFFFC22BDF501D
:10155000780AD8A4FBEF24F007808EC100F18FC178
:1015600001F190C102F191C103F10101040E046F78
:10157000000E056F000E066F000E076F9FEC28F03F
:1015800000AFCCEF0AF00101030E8E6F000E8F6FDB
:10159000000E906F000E916F03018251720AD8B451
:1015A000DCEF1FF08251520AD8B4DCEF1FF08251F9
:1015B000750AD8B4DCEF1FF08251630AD8B4B7EFD4
:1015C00021F08251690AD8B497EF1CF082517A0A4F
:1015D000D8B4AAEF1DF08251490AD8B436EF1CF0F6
:1015E0008251500AD8B454EF1BF08251700AD8B41B
:1015F00097EF1BF08251540AD8B4C2EF1BF082510E
:10160000740AD8B408EF1CF08251730AD8B40CEFF6
:101610001FF08251530AD8B471EF1FF082514C0A67
:10162000D8B402EF12F08251760AD8B42EEF0BF044
:10163000ECEF21F0040114EE00F080517F0BE12665
:1016400082C4E7FF802B120004010D0E826F1AEC9A
:101650000BF00A0E826F1AEC0BF01200030183519B
:10166000300AD8B4D3EF0CF003018351310AD8B457
:101670000AEF0DF003018351320AD8B4BFEF0EF028
:1016800003018351330AD8B474EF10F0030183517E
:10169000340AD8B41AEF11F003018351730AD8B495
:1016A000B5EF0BF003018351760AD8B4B7EF0BF016
:1016B00003018351740AD8B4A2EF0BF003018351E4
:1016C000540AD8B467EF0BF0D8A4ECEF21F0040172
:1016D000760E826F1AEC0BF00401540E826F1AEC36
:1016E0000BF007840001880E0C6EDBEC29F02981D9
:1016F000030184512D0AD8B480EF0BF00101299128
:1017000085C32FF186C330F187C331F188C332F12D
:1017100089C333F1E8EC29F05FEC29F000C10BF04C
:10172000DFEC07F001C10BF0DFEC07F0880EF6EC00
:1017300007F0E8CF40F6890EF6EC07F0E8CF41F667
:10174000ADEF0BF00401760E826F1AEC0BF0040182
:10175000740E826F1AEC0BF007840001880E0C6E79
:10176000FDEC07F0079401EF1AF0B5EC0BF0040163
:10177000760E826F1AEC0BF00401760E826F1AEC73
:101780000BF0078417EC26F004012C0E826F1AEC84
:101790000BF00101036B026B3BC601F13AC600F18D
:1017A00001AFD8EF0BF00101FF0E026FFF0E036FC8
:1017B0003DEC29F02967DFEF0BF0E4EF0BF00401BB
:1017C0002D0E826F1AEC0BF02FC182F40401300E43
:1017D00082271AEC0BF030C182F40401300E82270C
:1017E0001AEC0BF031C182F40401300E82271AEC9E
:1017F0000BF032C182F40401300E82271AEC0BF098
:1018000033C182F40401300E82271AEC0BF004017C
:101810002C0E826F1AEC0BF00101036B026B3DC6BC
:1018200001F13CC600F101AF1BEF0CF00101FF0E0E
:10183000026FFF0E036F3DEC29F0296722EF0CF0D9
:1018400027EF0CF004012D0E826F1AEC0BF02FC164
:1018500082F40401300E82271AEC0BF030C182F4BE
:101860000401300E82271AEC0BF031C182F404011E
:10187000300E82271AEC0BF032C182F40401300ED4
:1018800082271AEC0BF033C182F40401300E822758
:101890001AEC0BF004012C0E826F1AEC0BF0010114
:1018A000036B026B3FC601F13EC600F101AF5EEF74
:1018B0000CF00101FF0E026FFF0E036F3DEC29F0EB
:1018C000296765EF0CF06AEF0CF004012D0E826FB2
:1018D0001AEC0BF02FC182F40401300E82271AECAF
:1018E0000BF030C182F40401300E82271AEC0BF0A9
:1018F00031C182F40401300E82271AEC0BF032C1A0
:1019000082F40401300E82271AEC0BF033C182F40A
:101910000401300E82271AEC0BF004012C0E826FAA
:101920001AEC0BF00101036B026B37C601F136C6EE
:1019300000F101AFA1EF0CF00101FF0E026FFF0EED
:10194000036F3DEC29F02967A8EF0CF0ADEF0CF028
:1019500004012D0E826F1AEC0BF02FC182F40401EA
:10196000300E82271AEC0BF030C182F40401300EE5
:1019700082271AEC0BF031C182F40401300E822769
:101980001AEC0BF032C182F40401300E82271AECFB
:101990000BF033C182F40401300E82271AEC0BF0F5
:1019A000079401EF1AF00401760E826F1AEC0BF027
:1019B0000401300E826F1AEC0BF004012C0E826FC2
:1019C0001AEC0BF008EC2AF09AEC29F000C600F1B2
:1019D00001C601F13DEC29F030C182F40401300E62
:1019E00082271AEC0BF031C182F40401300E8227F9
:1019F0001AEC0BF032C182F40401300E82271AEC8B
:101A00000BF033C182F40401300E82271AEC0BF084
:101A100001EF1AF00401760E826F1AEC0BF004014C
:101A2000310E826F1AEC0BF007840101036B026B1D
:101A300002C600F103C601F101AF23EF0DF0FF0E66
:101A4000026FFF0E036F0101076B066B04C604F102
:101A500005C605F105AF31EF0DF0FF0E066FFF0E65
:101A6000076FA4EC28F00101076B066B06C604F1B2
:101A700007C605F105AF41EF0DF0FF0E066FFF0E33
:101A8000076FA4EC28F00101076B066B08C604F190
:101A900009C605F105AF51EF0DF0FF0E066FFF0E01
:101AA000076FA4EC28F0D89001010333023301330F
:101AB0000033D890010103330233013300330401B2
:101AC0002C0E826F1AEC0BF00101036B026B01C14B
:101AD00001F100C100F101AF73EF0DF00101FF0E44
:101AE000026FFF0E036F3DEC29F029677AEF0DF0CE
:101AF0007FEF0DF004012D0E826F1AEC0BF02FC159
:101B000082F40401300E82271AEC0BF030C182F40B
:101B10000401300E82271AEC0BF031C182F404016B
:101B2000300E82271AEC0BF032C182F40401300E21
:101B300082271AEC0BF033C182F40401300E8227A5
:101B40001AEC0BF00101036B026B0AC600F10BC625
:101B500001F101AFB0EF0DF0FF0E026FFF0E036F4A
:101B60000101076B066B0CC604F10DC605F105AF4C
:101B7000BEEF0DF0FF0E066FFF0E076FA4EC28F00E
:101B80000101076B066B0EC604F10FC605F105AF28
:101B9000CEEF0DF0FF0E066FFF0E076FA4EC28F0DE
:101BA0000101076B066B10C604F111C605F105AF04
:101BB000DEEF0DF0FF0E066FFF0E076FA4EC28F0AE
:101BC000D89001010333023301330033D89001016F
:101BD000033302330133003304012C0E826F1AECFD
:101BE0000BF00101036B026B01C101F100C100F1B7
:101BF00001AF00EF0EF00101FF0E026FFF0E036F49
:101C00003DEC29F0296707EF0EF00CEF0EF0040110
:101C10002D0E826F1AEC0BF02FC182F40401300EEE
:101C200082271AEC0BF030C182F40401300E8227B7
:101C30001AEC0BF031C182F40401300E82271AEC49
:101C40000BF032C182F40401300E82271AEC0BF043
:101C500033C182F40401300E82271AEC0BF001012B
:101C6000036B026B12C600F113C601F101AF3DEF29
:101C70000EF0FF0E026FFF0E036F0101076B066B84
:101C800014C604F115C605F105AF4BEF0EF0FF0EBB
:101C9000066FFF0E076FA4EC28F00101076B066BBF
:101CA00016C604F117C605F105AF5BEF0EF0FF0E87
:101CB000066FFF0E076FA4EC28F00101076B066B9F
:101CC00018C604F119C605F105AF6BEF0EF0FF0E53
:101CD000066FFF0E076FA4EC28F0D89001010333C4
:101CE000023301330033D89001010333023301334F
:101CF000003304012C0E826F1AEC0BF00101036B10
:101D0000026B01C101F100C100F101AF8DEF0EF0D6
:101D10000101FF0E026FFF0E036F3DEC29F02967F2
:101D200094EF0EF099EF0EF004012D0E826F1AEC75
:101D30000BF02FC182F40401300E82271AEC0BF055
:101D400030C182F40401300E82271AEC0BF031C14D
:101D500082F40401300E82271AEC0BF032C182F4B7
:101D60000401300E82271AEC0BF033C182F4040117
:101D7000300E82271AEC0BF0079401EF1AF00401E1
:101D8000760E826F1AEC0BF00401320E826F1AECA1
:101D90000BF007840101036B026B1AC600F11BC62E
:101DA00001F101AFD8EF0EF0FF0E026FFF0E036FCF
:101DB0000101076B066B1CC604F11DC605F105AFDA
:101DC000E6EF0EF0FF0E066FFF0E076FA4EC28F093
:101DD0000101076B066B1EC604F11FC605F105AFB6
:101DE000F6EF0EF0FF0E066FFF0E076FA4EC28F063
:101DF0000101076B066B20C604F121C605F105AF92
:101E000006EF0FF0FF0E066FFF0E076FA4EC28F031
:101E1000D89001010333023301330033D89001011C
:101E2000033302330133003304012C0E826F1AECAA
:101E30000BF00101036B026B01C101F100C100F164
:101E400001AF28EF0FF00101FF0E026FFF0E036FCD
:101E50003DEC29F029672FEF0FF034EF0FF004016C
:101E60002D0E826F1AEC0BF02FC182F40401300E9C
:101E700082271AEC0BF030C182F40401300E822765
:101E80001AEC0BF031C182F40401300E82271AECF7
:101E90000BF032C182F40401300E82271AEC0BF0F1
:101EA00033C182F40401300E82271AEC0BF00101D9
:101EB000036B026B22C600F123C601F101AF65EF8F
:101EC0000FF0FF0E026FFF0E036F0101076B066B31
:101ED00024C604F125C605F105AF73EF0FF0FF0E20
:101EE000066FFF0E076FA4EC28F00101076B066B6D
:101EF00026C604F127C605F105AF83EF0FF0FF0EEC
:101F0000066FFF0E076FA4EC28F00101076B066B4C
:101F100028C604F129C605F105AF93EF0FF0FF0EB7
:101F2000066FFF0E076FA4EC28F0D8900101033371
:101F3000023301330033D8900101033302330133FC
:101F4000003304012C0E826F1AEC0BF00101036BBD
:101F5000026B01C101F100C100F101AFB5EF0FF05B
:101F60000101FF0E026FFF0E036F3DEC29F02967A0
:101F7000BCEF0FF0C1EF0FF004012D0E826F1AECD1
:101F80000BF02FC182F40401300E82271AEC0BF003
:101F900030C182F40401300E82271AEC0BF031C1FB
:101FA00082F40401300E82271AEC0BF032C182F465
:101FB0000401300E82271AEC0BF033C182F40401C5
:101FC000300E82271AEC0BF00101036B026B2AC65C
:101FD00000F12BC601F101AFF2EF0FF0FF0E026F1F
:101FE000FF0E036F0101076B066B2CC604F12DC6B3
:101FF00005F105AF00EF10F0FF0E066FFF0E076F43
:10200000A4EC28F00101076B066B2EC604F12FC665
:1020100005F105AF10EF10F0FF0E066FFF0E076F12
:10202000A4EC28F00101076B066B30C604F131C641
:1020300005F105AF20EF10F0FF0E066FFF0E076FE2
:10204000A4EC28F0D89001010333023301330033AC
:10205000D8900101033302330133003304012C0E05
:10206000826F1AEC0BF00101036B026B01C101F1ED
:1020700000C100F101AF42EF10F00101FF0E026F4D
:10208000FF0E036F3DEC29F0296749EF10F04EEF8A
:1020900010F004012D0E826F1AEC0BF02FC182F4A8
:1020A0000401300E82271AEC0BF030C182F40401D7
:1020B000300E82271AEC0BF031C182F40401300E8D
:1020C00082271AEC0BF032C182F40401300E822711
:1020D0001AEC0BF033C182F40401300E82271AECA3
:1020E0000BF0079401EF1AF00401760E826F1AECE0
:1020F0000BF00401330E826F1AEC0BF004012C0E6E
:10210000826F1AEC0BF085C382F41AEC0BF0640EAC
:102110000D6E03018551320A02E16A0E0D6E030154
:102120008551330A02E1700E0D6E03018551340AA8
:1021300002E1760E0D6E03018551350A02E17C0E37
:102140000D6E03018551360A02E1820E0D6E030108
:102150008651780A65E00DC00CF0DBEC29F029818E
:10216000030187512D0AD8B4B8EF10F0010129916D
:1021700088C32FF189C330F18AC331F18BC332F1A7
:102180008CC333F1E8EC29F05FEC29F000C10BF0CF
:10219000DFEC07F001C10BF0DFEC07F0DBEC29F01E
:1021A000298103018E512D0AD8B4D9EF10F0010115
:1021B00029918FC32FF190C330F191C331F192C3B4
:1021C00032F193C333F1E8EC29F05FEC29F000C160
:1021D0000BF0DFEC07F001C10BF0DFEC07F0DBECFC
:1021E00029F02981030195512D0AD8B4FAEF10F096
:1021F0000101299196C32FF197C330F198C331F1B2
:1022000099C332F19AC333F1E8EC29F05FEC29F07D
:1022100000C10BF0DFEC07F001C10BF0DFEC07F0C1
:102220000DC00CF0FDEC07F0FDEC07F0FDEC07F045
:1022300001EF1AF00401760E826F1AEC0BF0040124
:10224000340E826F1AEC0BF003018451780AD8B473
:10225000F2EF11F03E0E0C6EDBEC29F02981030148
:1022600085512D0AD8B437EF11F00101299186C3A9
:102270002FF187C330F188C331F189C332F18AC3AA
:1022800033F1E8EC29F05FEC29F000C10BF0DFEC52
:1022900007F001C10BF0DFEC07F0DBEC29F029813E
:1022A00003018C512D0AD8B458EF11F00101299186
:1022B0008DC32FF18EC330F18FC331F190C332F152
:1022C00091C333F1E8EC29F05FEC29F000C10BF089
:1022D000DFEC07F001C10BF0DFEC07F0DBEC29F0DD
:1022E0002981030193512D0AD8B479EF11F001012E
:1022F000299194C32FF195C330F196C331F197C35F
:1023000032F198C333F1E8EC29F05FEC29F000C119
:102310000BF0DFEC07F001C10BF0DFEC07F0DBECBA
:1023200029F0298103019A512D0AD8B49AEF11F0AE
:10233000010129919BC32FF19CC330F19DC331F161
:102340009EC332F19FC333F1E8EC29F05FEC29F032
:1023500000C10BF0DFEC07F001C10BF0DFEC07F080
:10236000DBEC29F029810301A1512D0AD8B4BBEF80
:1023700011F001012991A2C32FF1A3C330F1A4C32D
:1023800031F1A5C332F1A6C333F1E8EC29F05FECDB
:1023900029F000C10BF0DFEC07F001C10BF0DFEC1E
:1023A00007F0DBEC29F029810301A8512D0AD8B4EC
:1023B000DCEF11F001012991A9C32FF1AAC330F17B
:1023C000ABC331F1ACC332F1ADC333F1E8EC29F06A
:1023D0005FEC29F000C10BF0DFEC07F001C10BF05E
:1023E000DFEC07F03E0E0C6EFDEC07F0FDEC07F0A5
:1023F000FDEC07F0FDEC07F0FDEC07F0FDEC07F05D
:1024000001EF1AF003018351300AD8B4C3EF14F07E
:1024100003018351310AD8B4D1EF15F00301835180
:10242000320AD8B43FEF16F003018351330AD8B40F
:102430004FEF16F003018351340AD8B45FEF16F062
:1024400003018351350AD8B4A5EF19F00301835174
:10245000360AD8B4D3EF19F003018351460AD8B431
:10246000F9EF18F0030183514D0AD8B43CEF13F093
:10247000030183516D0AD8B456EF13F00301835161
:102480005A0AD8B44BEF15F003018351490AD8B466
:10249000D3EF1AF003018351500AD8B405EF1AF0B4
:1024A00003018351540AD8B47EEF1AF0030183511B
:1024B000630AD8B476EF13F003018351430AD8B40A
:1024C0006EEF14F003018351730AD8B474EF13F064
:1024D00003018351610AD8B489EF12F003018351DB
:1024E000650AD8B413EF15F003018351450AD8B437
:1024F00021EF15F003018351620AD8B42FEF15F0D4
:1025000003018351420AD8B43DEF15F0D8A4ECEF93
:1025100021F004014C0E826F1AEC0BF00401610EE5
:10252000826F1AEC0BF003EC2CF004012C0E826F7E
:102530001AEC0BF09AEC29F0ABC500F101013DEC6F
:1025400029F031C182F40401300E82271AEC0BF01D
:1025500032C182F40401300E82271AEC0BF033C131
:1025600082F40401300E82271AEC0BF004012C0EC9
:10257000826F1AEC0BF09AEC29F0ACC500F1010166
:102580003DEC29F031C182F40401300E82271AECAF
:102590000BF032C182F40401300E82271AEC0BF0EA
:1025A00033C182F40401300E82271AEC0BF00401CF
:1025B0002C0E826F1AEC0BF09AEC29F0ADC500F1ED
:1025C00001013DEC29F031C182F40401300E822773
:1025D0001AEC0BF032C182F40401300E82271AEC9F
:1025E0000BF033C182F40401300E82271AEC0BF099
:1025F00004012C0E826F1AEC0BF09AEC29F0AEC598
:1026000000F101013DEC29F031C182F40401300EEA
:1026100082271AEC0BF032C182F40401300E8227BB
:102620001AEC0BF033C182F40401300E82271AEC4D
:102630000BF004012C0E826F1AEC0BF09AEC29F0CF
:10264000B3C500F101013DEC29F031C182F4040170
:10265000300E82271AEC0BF032C182F40401300EE6
:1026600082271AEC0BF033C182F40401300E82276A
:102670001AEC0BF001EF1AF0DBEC29F084C333F114
:10268000E8EC29F05FEC29F0200E0C6E00C10BF095
:10269000DFEC07F000C12FF505012F51000A06E01D
:1026A00005012F51010A02E0A9EC2CF004014C0EA7
:1026B000826F1AEC0BF004014D0E826F1AEC0BF0D6
:1026C00004012C0E826F1AEC0BF09AEC29F02FC546
:1026D00000F13DEC29F033C182F40401300E822771
:1026E0001AEC0BF001EF1AF0C0EF33F004014C0EBE
:1026F000826F1AEC0BF00401630E826F1AEC0BF080
:1027000053EC2BF004012C0E826F1AEC0BF08BECC7
:1027100013F001EF1AF09AEC29F0B1C500F10101B4
:10272000003B0F0E00173DEC29F033C182F4040189
:10273000300E82271AEC0BF0B1C500F101010F0E2B
:10274000010100173DEC29F033C182F40401300E81
:1027500082271AEC0BF004012D0E826F1AEC0BF09D
:10276000B0C500F10101003B0F0E00173DEC29F050
:1027700033C182F40401300E82271AEC0BF0B0C58D
:1027800000F101010F0E010100173DEC29F033C1EA
:1027900082F40401300E82271AEC0BF004012D0E96
:1027A000826F1AEC0BF0AFC500F10101003B0F0E78
:1027B00000173DEC29F033C182F40401300E82276A
:1027C0001AEC0BF0AFC500F101010F0E010100176B
:1027D0003DEC29F033C182F40401300E82271AEC5B
:1027E0000BF00401200E826F1AEC0BF0AEC500F165
:1027F0000F0E010100173DEC29F033C182F40401F2
:10280000300E82271AEC0BF00401200E826F1AECB6
:102810000BF0ADC500F101010101003B0F0E0017E7
:102820003DEC29F033C182F40401300E82271AEC0A
:102830000BF0ADC500F101010F0E010100173DECD9
:1028400029F033C182F40401300E82271AEC0BF018
:1028500004013A0E826F1AEC0BF0ACC500F10101D5
:10286000003B0F0E00173DEC29F033C182F4040148
:10287000300E82271AEC0BF0ACC500F101010F0EEF
:10288000010100173DEC29F033C182F40401300E40
:1028900082271AEC0BF004013A0E826F1AEC0BF04F
:1028A000ABC500F10101003B0F0E00173DEC29F014
:1028B00033C182F40401300E82271AEC0BF0ABC551
:1028C00000F101010F0E00173DEC29F033C182F435
:1028D0000401300E82271AEC0BF0120084C3E8FFCB
:1028E0000F0BE83AE8CFB1F585C3E8FF0F0B050100
:1028F000B11387C3E8FF0F0BE83AE8CFB0F588C300
:10290000E8FF0F0B0501B0138AC3E8FF0F0BE83A8D
:10291000E8CFAFF58BC3E8FF0F0B0501AF138DC3F5
:10292000E8FF0F0BE8CFAEF58FC3E8FF0F0BE83AD7
:10293000E8CFADF590C3E8FF0F0B0501AD1392C3CF
:10294000E8FF0F0BE83AE8CFACF593C3E8FF0F0BB5
:102950000501AC1395C3E8FF0F0BE83AE8CFABF5E0
:1029600096C3E8FF0F0B0501AB13B2EC2BF004018B
:102970004C0E826F1AEC0BF00401430E826F1AECBE
:102980000BF080EF13F0078481EC33F09AEC29F020
:102990002DC500F13DEC29F004014C0E826F1AECBC
:1029A0000BF00401300E826F1AEC0BF004012C0EB8
:1029B000826F1AEC0BF031C182F40401300E8227D1
:1029C0001AEC0BF032C182F40401300E82271AECAB
:1029D0000BF033C182F40401300E82271AEC0BF0A5
:1029E00004012C0E826F1AEC0BF09AEC29F02EC524
:1029F00000F13DEC29F031C182F40401300E822750
:102A00001AEC0BF032C182F40401300E82271AEC6A
:102A10000BF033C182F40401300E82271AEC0BF064
:102A2000079401EF1AF004014C0E826F1AEC0BF0C0
:102A30000401650E826F1AEC0BF092EC2DF001EFA1
:102A40001AF004014C0E826F1AEC0BF00401450ED3
:102A5000826F1AEC0BF0AFEC2DF001EF1AF00401CD
:102A60004C0E826F1AEC0BF00401620E826F1AECAE
:102A70000BF0E9EC2DF001EF1AF004014C0E826F1F
:102A80001AEC0BF00401420E826F1AEC0BF0CCEC46
:102A90002DF001EF1AF004014C0E826F1AEC0BF0CE
:102AA00004015A0E826F1AEC0BF004012C0E826F97
:102AB0001AEC0BF081EC33F09AEC29F005012E5161
:102AC000130A06E005012E51170A0DE07CEF15F000
:102AD0000101000E006F000E016F100E026F000E5C
:102AE000036F7CEF15F00101000E006F000E016F07
:102AF000000E026F010E036F0101200E046F000E25
:102B0000056F000E066F000E076FD0EC28F03DEC4D
:102B100029F02AC182F40401300E82271AEC0BF04E
:102B20002BC182F40401300E82271AEC0BF02CC169
:102B300082F40401300E82271AEC0BF02DC182F4CE
:102B40000401300E82271AEC0BF02EC182F404012E
:102B5000300E82271AEC0BF02FC182F40401300EE4
:102B600082271AEC0BF030C182F40401300E822768
:102B70001AEC0BF031C182F40401300E82271AECFA
:102B80000BF032C182F40401300E82271AEC0BF0F4
:102B900033C182F40401300E82271AEC0BF001EFEE
:102BA0001AF0078404014C0E826F1AEC0BF004013A
:102BB000310E826F1AEC0BF004012C0E826F1AECAE
:102BC0000BF025C500F126C501F127C502F128C586
:102BD00003F10101200E046F000E056F000E066F59
:102BE000000E076FD0EC28F03DEC29F02AC182F4EA
:102BF0000401300E82271AEC0BF02BC182F4040181
:102C0000300E82271AEC0BF02CC182F40401300E36
:102C100082271AEC0BF02DC182F40401300E8227BA
:102C20001AEC0BF02EC182F40401300E82271AEC4C
:102C30000BF02FC182F40401300E82271AEC0BF046
:102C400030C182F40401300E82271AEC0BF031C13E
:102C500082F40401300E82271AEC0BF032C182F4A8
:102C60000401300E82271AEC0BF033C182F4040108
:102C7000300E82271AEC0BF0079401EF1AF007844C
:102C800004014C0E826F1AEC0BF00401320E826FBD
:102C90001AEC0BF0DFEC2FF0079401EF1AF0078429
:102CA00004014C0E826F1AEC0BF00401330E826F9C
:102CB0001AEC0BF03CEC30F00794DCEF15F00784D5
:102CC00004014C0E826F1AEC0BF00401340E826F7B
:102CD0001AEC0BF004012C0E826F1AEC0BF0DBECFB
:102CE00029F084C32AF185C32BF186C32CF187C355
:102CF0002DF188C32EF189C32FF18AC330F18BC324
:102D000031F18CC332F18DC333F10101296BE8EC51
:102D100029F05FEC29F0200E046F000E056F000E05
:102D2000066F000E076FB0EC28F000C121F501C15D
:102D300022F502C123F503C124F534EC33F034C588
:102D4000ABF535C5ACF536C5ADF537C5AEF538C50F
:102D5000AFF539C5B0F53AC5B1F58BEC13F0040108
:102D60002C0E826F1AEC0BF03BC500F13CC501F153
:102D70003DC502F13EC503F10101000E046F000ED6
:102D8000056F010E066F000E076FD0EC28F03DECCA
:102D900029F02967CEEF16F0D3EF16F004012D0EBF
:102DA000826F1AEC0BF030C182F40401300E8227DE
:102DB0001AEC0BF031C182F40401300E82271AECB8
:102DC0000BF004012E0E826F1AEC0BF032C182F46C
:102DD0000401300E82271AEC0BF033C182F4040197
:102DE000300E82271AEC0BF004012C0E826F1AECC5
:102DF0000BF09AEC29F03FC500F140C501F116EC4B
:102E000023F004012C0E826F1AEC0BF09AEC29F0DF
:102E100041C500F13DEC29F031C182F40401300ECE
:102E200082271AEC0BF032C182F40401300E8227A3
:102E30001AEC0BF033C182F40401300E82271AEC35
:102E40000BF004012C0E826F1AEC0BF00101036BE6
:102E5000026B48C501F147C500F101AF35EF17F02E
:102E60000101FF0E026FFF0E036F3DEC29F0296791
:102E70003CEF17F041EF17F004012D0E826F1AECB2
:102E80000BF02FC182F40401300E82271AEC0BF0F4
:102E900030C182F40401300E82271AEC0BF031C1EC
:102EA00082F40401300E82271AEC0BF032C182F456
:102EB0000401300E82271AEC0BF033C182F40401B6
:102EC000300E82271AEC0BF004012C0E826F1AECE4
:102ED0000BF00101036B026B4AC501F149C500F11A
:102EE00001AF78EF17F00101FF0E026FFF0E036FC5
:102EF0003DEC29F029677FEF17F084EF17F004010C
:102F00002D0E826F1AEC0BF02FC182F40401300EEB
:102F100082271AEC0BF030C182F40401300E8227B4
:102F20001AEC0BF031C182F40401300E82271AEC46
:102F30000BF032C182F40401300E82271AEC0BF040
:102F400033C182F40401300E82271AEC0BF0040125
:102F50002C0E826F1AEC0BF00101036B026B4CC557
:102F600001F14BC500F101AFBBEF17F00101FF0EFE
:102F7000026FFF0E036F3DEC29F02967C2EF17F0D7
:102F8000C7EF17F004012D0E826F1AEC0BF02FC162
:102F900082F40401300E82271AEC0BF030C182F467
:102FA0000401300E82271AEC0BF031C182F40401C7
:102FB000300E82271AEC0BF032C182F40401300E7D
:102FC00082271AEC0BF033C182F40401300E822701
:102FD0001AEC0BF004012C0E826F1AEC0BF00101BD
:102FE000036B026B4EC501F14DC500F101AFFEEF61
:102FF00017F00101FF0E026FFF0E036F3DEC29F089
:10300000296705EF18F00AEF18F004012D0E826F02
:103010001AEC0BF02FC182F40401300E82271AEC57
:103020000BF030C182F40401300E82271AEC0BF051
:1030300031C182F40401300E82271AEC0BF032C148
:1030400082F40401300E82271AEC0BF033C182F4B3
:103050000401300E82271AEC0BF004012C0E826F53
:103060001AEC0BF00101036B026B50C501F14FC567
:1030700000F101AF41EF18F00101FF0E026FFF0EEA
:10308000036F3DEC29F0296748EF18F04DEF18F079
:1030900004012D0E826F1AEC0BF02FC182F4040193
:1030A000300E82271AEC0BF030C182F40401300E8E
:1030B00082271AEC0BF031C182F40401300E822712
:1030C0001AEC0BF032C182F40401300E82271AECA4
:1030D0000BF033C182F40401300E82271AEC0BF09E
:1030E00004012C0E826F1AEC0BF00101036B026BD2
:1030F00052C501F151C500F101AF84EF18F0010193
:10310000FF0E026FFF0E036F3DEC29F029678BEF76
:1031100018F090EF18F004012D0E826F1AEC0BF0EE
:103120002FC182F40401300E82271AEC0BF030C15B
:1031300082F40401300E82271AEC0BF031C182F4C4
:103140000401300E82271AEC0BF032C182F4040124
:10315000300E82271AEC0BF033C182F40401300EDA
:1031600082271AEC0BF004012C0E826F1AEC0BF084
:103170000101036B026B46C501F145C500F101AFCA
:10318000C7EF18F00101FF0E026FFF0E036F3DEC59
:1031900029F02967CEEF18F0D3EF18F004012D0EB7
:1031A000826F1AEC0BF02FC182F40401300E8227DB
:1031B0001AEC0BF030C182F40401300E82271AECB5
:1031C0000BF031C182F40401300E82271AEC0BF0AF
:1031D00032C182F40401300E82271AEC0BF033C1A5
:1031E00082F40401300E82271AEC0BF0079401EFF1
:1031F0001AF0DBEC29F085C32AF186C32BF187C3D3
:103200002CF188C32DF189C32EF18AC32FF18BC312
:1032100030F18CC331F18DC332F18EC333F1010132
:10322000296BE8EC29F05FEC29F00101010E046F35
:10323000000E056F000E066F000E076F9FEC28F062
:10324000100E046F000E056F000E066F000E076F64
:10325000B0EC28F000C129F501C12AF502C12BF517
:1032600003C12CF568EC2FF004014C0E826F1AECB0
:103270000BF00401460E826F1AEC0BF004012C0EC9
:10328000826F1AEC0BF025C500F126C501F127C5A8
:1032900002F128C503F10101100E046F000E056F45
:1032A000000E066F000E076FD0EC28F03DEC29F001
:1032B0002AC182F40401300E82271AEC0BF02BC1D4
:1032C00082F40401300E82271AEC0BF02CC182F438
:1032D0000401300E82271AEC0BF02DC182F4040198
:1032E000300E82271AEC0BF02EC182F40401300E4E
:1032F00082271AEC0BF02FC182F40401300E8227D2
:103300001AEC0BF030C182F40401300E82271AEC63
:103310000BF031C182F40401300E82271AEC0BF05D
:1033200032C182F40401300E82271AEC0BF033C153
:1033300082F40401300E82271AEC0BF001EF1AF030
:103340000F983CEC30F0ECEF21F004014C0E826F52
:103350001AEC0BF00401350E826F1AEC0BF004012D
:103360002C0E826F1AEC0BF09AEC29F00784B5C58D
:1033700000F107943DEC29F031C182F40401300ED4
:1033800082271AEC0BF032C182F40401300E82273E
:103390001AEC0BF033C182F40401300E82271AECD0
:1033A0000BF001EF1AF0FFEC2FF09AEC29F033C587
:1033B00000F13DEC29F004014C0E826F1AEC0BF089
:1033C0000401360E826F1AEC0BF004012C0E826F92
:1033D0001AEC0BF031C182F40401300E82271AEC92
:1033E0000BF032C182F40401300E82271AEC0BF08C
:1033F00033C182F40401300E82271AEC0BF001EF86
:103400001AF024EC0BF0ECEF21F004014C0E826F6B
:103410001AEC0BF00401500E826F1AEC0BF0040151
:103420002C0E826F1AEC0BF085C32AF186C32BF1A8
:1034300087C32CF188C32DF189C32EF18AC32FF1E4
:103440008BC330F18CC331F18DC332F18EC333F1B4
:103450000101E8EC29F05FEC29F003018451530AE3
:103460000DE0030184514D0A38E00401780E826FAB
:103470001AEC0BF024EC0BF0ECEF21F00401530EEE
:10348000826F1AEC0BF0250E0C6E00C10BF0DFEC16
:1034900007F0260E0C6E01C10BF0DFEC07F0270ED3
:1034A0000C6E02C10BF0DFEC07F0280E0C6E03C1AE
:1034B0000BF0DFEC07F000C153F501C154F502C178
:1034C00055F503C156F500C157F501C158F502C1C4
:1034D00059F503C15AF5E2EF1AF004014D0E826F5F
:1034E0001AEC0BF0290E0C6E00C10BF0DFEC07F0AC
:1034F00000C15BF500C15CF5E2EF1AF004014C0E6F
:10350000826F1AEC0BF00401540E826F1AEC0BF070
:1035100004012C0E826F1AEC0BF084C32AF185C3D0
:103520002BF186C32CF187C32DF188C32EF189C3FB
:103530002FF18AC330F18BC331F18DC332F18EC3C9
:1035400033F10101E8EC29F05FEC29F00101000EF4
:10355000046F000E056F010E066F000E076FB0ECD2
:1035600028F0210E0C6E00C10BF0DFEC07F0220EEC
:103570000C6E01C10BF0DFEC07F0230E0C6E02C1E4
:103580000BF0DFEC07F0240E0C6E03C10BF0DFEC48
:1035900007F000C15DF501C15EF502C15FF503C131
:1035A00060F5E2EF1AF004014C0E826F1AEC0BF09A
:1035B0000401490E826F1AEC0BF004012C0E826F8D
:1035C0001AEC0BF0250EF6EC07F0E8CF00F1260E12
:1035D000F6EC07F0E8CF01F1270EF6EC07F0E8CFA4
:1035E00002F1280EF6EC07F0E8CF03F13DEC29F0EC
:1035F00020EC27F00401730E826F1AEC0BF004012B
:103600002C0E826F1AEC0BF09AEC29F0290EF6ECD6
:1036100007F0E8CF00F13DEC29F020EC27F00401A1
:10362000730E826F1AEC0BF004012C0E826F1AECF1
:103630000BF057C500F158C501F159C502F15AC543
:1036400003F13DEC29F020EC27F00401730E826FAA
:103650001AEC0BF004012C0E826F1AEC0BF09AECB2
:1036600029F05CC500F13DEC29F020EC27F00401C5
:103670006D0E826F1AEC0BF004012C0E826F1AECA7
:103680000BF05DC500F15EC501F15FC502F160C5DB
:1036900003F107EC22F004012C0E826F1AEC0BF000
:1036A00024EC0BF0ECEF21F083C32AF184C32BF15F
:1036B00085C32CF186C32DF187C32EF188C32FF16A
:1036C00089C330F18AC331F18BC332F18CC333F13A
:1036D0000101E8EC29F05FEC29F0160E0C6E00C138
:1036E0000BF0DFEC07F0170E0C6E01C10BF0DFECF6
:1036F00007F0180E0C6E02C10BF0DFEC07F0190E8C
:103700000C6E03C10BF0DFEC07F000C18AF101C1C0
:103710008BF102C18CF103C18DF100C18EF101C1A9
:103720008FF102C190F103C191F136EF1CF083C318
:103730002AF184C32BF185C32CF186C32DF187C3F5
:103740002EF188C32FF189C330F18AC331F18BC3C5
:1037500032F18CC333F10101E8EC29F05FEC29F080
:1037600000C18AF101C18BF102C18CF103C18DF15D
:1037700000C18EF101C18FF102C190F103C191F13D
:1037800036EF1CF083C32AF184C32BF185C32CF1DF
:1037900086C32DF187C32EF188C32FF189C330F181
:1037A0008AC331F18CC332F18DC333F10101E8ECEE
:1037B00029F05FEC29F00101000E046F000E056F87
:1037C000010E066F000E076FB0EC28F01A0E0C6E9B
:1037D00000C10BF0DFEC07F01B0E0C6E01C10BF00B
:1037E000DFEC07F01C0E0C6E02C10BF0DFEC07F0F3
:1037F0001D0E0C6E03C10BF0DFEC07F000C192F15F
:1038000001C193F102C194F103C195F136EF1CF0AF
:1038100083C32AF184C32BF185C32CF186C32DF118
:1038200087C32EF188C32FF189C330F18AC331F1E8
:103830008CC332F18DC333F10101E8EC29F05FEC68
:1038400029F00101000E046F000E056F010E066FD6
:10385000000E076FB0EC28F000C192F101C193F1A6
:1038600002C194F103C195F136EF1CF0160EF6EC8F
:1038700007F0E8CF00F1170EF6EC07F0E8CF01F102
:10388000180EF6EC07F0E8CF02F1190EF6EC07F08F
:10389000E8CF03F13DEC29F020EC27F00401730E92
:1038A000826F1AEC0BF004012C0E826F1AEC0BF0F5
:1038B0008AC100F18BC101F18CC102F18DC103F10C
:1038C0003DEC29F020EC27F00401730E826F1AEC16
:1038D0000BF004012C0E826F1AEC0BF01A0EF6ECB2
:1038E00007F0E8CF00F11B0EF6EC07F0E8CF01F18E
:1038F0001C0EF6EC07F0E8CF02F11D0EF6EC07F017
:10390000E8CF03F107EC22F004012C0E826F1AECD1
:103910000BF092C100F193C101F194C102F195C184
:1039200003F107EC22F024EC0BF0ECEF21F00401A2
:10393000690E826F1AEC0BF004012C0E826F1AECE8
:103940000BF00101040E006F000E016F000E026FFC
:10395000000E036F3DEC29F02CC182F40401300EFF
:1039600082271AEC0BF02DC182F40401300E82275D
:103970001AEC0BF02EC182F40401300E82271AECEF
:103980000BF02FC182F40401300E82271AEC0BF0E9
:1039900030C182F40401300E82271AEC0BF031C1E1
:1039A00082F40401300E82271AEC0BF032C182F44B
:1039B0000401300E82271AEC0BF033C182F40401AB
:1039C000300E82271AEC0BF004012C0E826F1AECD9
:1039D0000BF001010B0E006F000E016F000E026F65
:1039E000000E036F3DEC29F02CC182F40401300E6F
:1039F00082271AEC0BF02DC182F40401300E8227CD
:103A00001AEC0BF02EC182F40401300E82271AEC5E
:103A10000BF02FC182F40401300E82271AEC0BF058
:103A200030C182F40401300E82271AEC0BF031C150
:103A300082F40401300E82271AEC0BF032C182F4BA
:103A40000401300E82271AEC0BF033C182F404011A
:103A5000300E82271AEC0BF004012C0E826F1AEC48
:103A60000BF00101210E006F000E016F000E026FBE
:103A7000000E036F3DEC29F02CC182F40401300EDE
:103A800082271AEC0BF02DC182F40401300E82273C
:103A90001AEC0BF02EC182F40401300E82271AECCE
:103AA0000BF02FC182F40401300E82271AEC0BF0C8
:103AB00030C182F40401300E82271AEC0BF031C1C0
:103AC00082F40401300E82271AEC0BF032C182F42A
:103AD0000401300E82271AEC0BF033C182F404018A
:103AE000300E82271AEC0BF004012C0E826F1AECB8
:103AF0000BF0200EF86EF76AF66A04010900F5CFA4
:103B000082F41AEC0BF00900F5CF82F41AEC0BF0FA
:103B10000900F5CF82F41AEC0BF00900F5CF82F41E
:103B20001AEC0BF00900F5CF82F41AEC0BF0090047
:103B3000F5CF82F41AEC0BF00900F5CF82F41AEC01
:103B40000BF00900F5CF82F41AEC0BF024EC0BF02B
:103B5000ECEF21F08351630AD8A4ECEF21F08451FB
:103B6000610AD8A4ECEF21F085516C0AD8A4ECEFDF
:103B700021F08651410A42E08651440A1BE08651F9
:103B8000420AD8B411EF1EF08651350AD8B476EF48
:103B900023F08651360AD8B4CBEF23F08651370A8A
:103BA000D8B434EF24F08651380AD8B492EF24F018
:103BB000ECEF21F00798079A04017A0E826F1AEC55
:103BC0000BF00401780E826F1AEC0BF00401640E06
:103BD000826F1AEC0BF081A8F5EF1DF00401550E71
:103BE000826F1AEC0BF0FAEF1DF004014C0E826F9D
:103BF0001AEC0BF024EC0BF0ECEF21F00788079A9D
:103C000004017A0E826F1AEC0BF00401410E826FF0
:103C10001AEC0BF00401610E826F1AEC0BF0EBEF63
:103C20001DF00798078A04017A0E826F1AEC0BF0D8
:103C30000401420E826F1AEC0BF00401610E826FD8
:103C40001AEC0BF0EBEF1DF0010166672FEF1EF091
:103C500067672FEF1EF068672FEF1EF0696747EF69
:103C60001EF04F673BEF1EF050673BEF1EF05167B1
:103C70003BEF1EF0526747EF1EF00101000E006F90
:103C8000000E016F000E026F000E036F12000101A3
:103C9000620E046F010E056F000E066F000E076FB7
:103CA00066C100F167C101F168C102F169C103F1A8
:103CB0009FEC28F003BFCBEF1EF00101000E046F54
:103CC000A80E056F550E066F020E076F66C100F154
:103CD00067C101F168C102F169C103F166C186F1F2
:103CE00067C187F168C188F169C189F19FEC28F04B
:103CF00003BF84EF1EF00101000E866FA80E876FD0
:103D0000550E886F020E896F0E0EF6EC07F0E8CFA5
:103D100018F10F0EF6EC07F0E8CF19F1100EF6ECE3
:103D200007F0E8CF1AF1110EF6EC07F0E8CF1BF11F
:103D3000E8EC27F086C104F187C105F188C106F1DE
:103D400089C107F19FEC28F00782ACEC27F0E8EC82
:103D500027F00792ACEC27F086C100F187C101F192
:103D600088C102F189C103F10792ACEC27F0CC0EB7
:103D7000046FE00E056F870E066F050E076F9FEC50
:103D800028F000C118F101C119F102C11AF103C1F3
:103D90001BF103EF1FF00101800E006F1A0E016F7F
:103DA000060E026F000E036F4FC104F150C105F102
:103DB00051C106F152C107F19FEC28F003AFE4EFC7
:103DC0001EF09AEC29F012000E0EF6EC07F0E8CF88
:103DD00018F10F0EF6EC07F0E8CF19F1100EF6EC23
:103DE00007F0E8CF1AF1110EF6EC07F0E8CF1BF15F
:103DF0004FC100F150C101F151C102F152C103F1B3
:103E00000782ACEC27F018C100F119C101F11AC109
:103E100002F11BC103F112000401730E826F1AEC50
:103E20000BF004012C0E826F1AEC0BF0078462C1B8
:103E300066F163C167F164C168F165C169F14BC1A5
:103E40004FF14CC150F14DC151F14EC152F157C12A
:103E500059F158C15AF1079432EC1FF024EC0BF0E1
:103E6000ECEF21F066C100F167C101F168C102F118
:103E700069C103F101013DEC29F020EC27F00401B8
:103E8000630E826F1AEC0BF004012C0E826F1AEC99
:103E90000BF04FC100F150C101F151C102F152C10B
:103EA00003F101013DEC29F020EC27F00401660E3E
:103EB000826F1AEC0BF004012C0E826F1AEC0BF0DF
:103EC0009AEC29F059C100F15AC101F101013DEC10
:103ED00029F020EC27F00401740E826F1AEC0BF02D
:103EE000120010820401530E826F1AEC0BF00401D1
:103EF0002C0E826F1AEC0BF083C32AF184C32BF1D2
:103F000085C32CF186C32DF187C32EF188C32FF111
:103F100089C330F18AC331F18BC332F18CC333F1E1
:103F20000101E8EC29F05FEC29F000C166F101C164
:103F300067F102C168F103C169F18EC32AF18FC331
:103F40002BF190C32CF191C32DF192C32EF193C3A9
:103F50002FF194C330F195C331F196C332F197C379
:103F600033F10101E8EC29F05FEC29F000C14FF1D9
:103F700001C150F102C151F103C152F1DBEC29F052
:103F800099C32FF19AC330F19BC331F19CC332F135
:103F90009DC333F10101E8EC29F05FEC29F000C189
:103FA00059F101C15AF132EC1FF004012C0E826F5D
:103FB0001AEC0BF0E3EF1FF08251520A03E10F827B
:103FC000E3EF1FF00F928251750A03E11084EAEFCC
:103FD0001FF010948251550A03E11086F1EF1FF093
:103FE0001096078410B24EEF20F010A43AEF20F0A4
:103FF000B6C166F1B7C167F1B8C168F1B9C169F17D
:10400000BAC16AF1BBC16BF1BCC16CF1BDC16DF14C
:10401000BEC16EF1BFC16FF1C0C170F1C1C171F11C
:10402000C2C172F1C3C173F1C4C174F1C5C175F1EC
:10403000C6C176F1C7C177F1C8C178F1C9C179F1BC
:10404000CAC17AF1CBC17BF1CCC17CF1CDC17DF18C
:10405000CEC17EF1CFC17FF1D0C180F1D1C181F15C
:10406000D2C182F1D3C183F1D4C184F1D5C185F12C
:1040700042EF20F062C166F163C167F164C168F18B
:1040800065C169F14BC14FF14CC150F14DC151F1C6
:104090004EC152F157C159F158C15AF107940FA0BE
:1040A00070EF20F0010192675DEF20F093675DEF04
:1040B00020F094675DEF20F0956761EF20F070EFDE
:1040C00020F024EC1EF092C104F193C105F194C1DB
:1040D00006F195C107F19FEC28F003BFB4EF21F082
:1040E00024EC1EF00101000E046F000E056F010E9E
:1040F000066F000E076FD0EC28F010A487EF20F0B9
:104100000401750E826F1AEC0BF08CEF20F00401A5
:10411000720E826F1AEC0BF004012C0E826F1AECF7
:104120000BF03DEC29F029679BEF20F00401200EF5
:10413000826F9EEF20F004012D0E826F1AEC0BF0BF
:1041400030C182F40401300E82271AEC0BF031C129
:1041500082F40401300E82271AEC0BF004012E0EBB
:10416000826F1AEC0BF032C182F40401300E822708
:104170001AEC0BF033C182F40401300E82271AECE2
:104180000BF004016D0E826F1AEC0BF004012C0E83
:10419000826F1AEC0BF04FC100F150C101F151C117
:1041A00002F152C103F101013DEC29F020EC27F0AE
:1041B0000401480E826F1AEC0BF004017A0E826F34
:1041C0001AEC0BF004012C0E826F1AEC0BF066C196
:1041D00000F167C101F168C102F169C103F1010198
:1041E0003DEC29F020EC27F00401630E826F1AECFD
:1041F0000BF004012C0E826F1AEC0BF066C100F17B
:1042000067C101F168C102F169C103F101010A0E40
:10421000046F000E056F000E066F000E076FB0EC06
:1042200028F0000E046F120E056F000E066F000ED0
:10423000076FD0EC28F03DEC29F02AC182F404018C
:10424000300E82271AEC0BF02BC182F40401300EE1
:1042500082271AEC0BF02CC182F40401300E822765
:104260001AEC0BF02DC182F40401300E82271AECF7
:104270000BF02EC182F40401300E82271AEC0BF0F1
:104280002FC182F40401300E82271AEC0BF030C1EA
:1042900082F40401300E82271AEC0BF004012E0E7A
:1042A000826F1AEC0BF031C182F40401300E8227C8
:1042B0001AEC0BF032C182F40401300E82271AECA2
:1042C0000BF033C182F40401300E82271AEC0BF09C
:1042D0000401730E826F1AEC0BF004012C0E826F36
:1042E0001AEC0BF09AEC29F059C100F15AC101F116
:1042F00016EC23F00FB280EF21F00FA0B2EF21F007
:1043000004012C0E826F1AEC0BF0200EF86EF76A87
:10431000F66A04010900F5CF82F41AEC0BF00900EB
:10432000F5CF82F41AEC0BF00900F5CF82F41AEC09
:104330000BF00900F5CF82F41AEC0BF00900F5CF71
:1043400082F41AEC0BF00900F5CF82F41AEC0BF0B2
:104350000900F5CF82F41AEC0BF00900F5CF82F4D6
:104360001AEC0BF024EC0BF00F90ECEF21F00401B1
:10437000630E826F1AEC0BF004012C0E826F1AECA4
:104380000BF0F2EC21F004012C0E826F1AEC0BF012
:1043900065EC22F004012C0E826F1AEC0BF0E1ECBC
:1043A00022F004012C0E826F1AEC0BF00101F80EC2
:1043B000006FCD0E016F660E026F030E036F07ECE8
:1043C00022F004012C0E826F1AEC0BF0F7EC22F0B5
:1043D00024EC0BF0ECEF21F00301C26B079010927C
:1043E000FBEF24F0D8900E0EF6EC07F0E8CF00F1CA
:1043F0000F0EF6EC07F0E8CF01F1100EF6EC07F027
:10440000E8CF02F1110EF6EC07F0E8CF03F101015D
:10441000000E046F000E056F010E066F000E076F91
:10442000D0EC28F03DEC29F02AC182F40401300ED2
:1044300082271AEC0BF02BC182F40401300E822784
:104440001AEC0BF02CC182F40401300E82271AEC16
:104450000BF02DC182F40401300E82271AEC0BF010
:104460002EC182F40401300E82271AEC0BF02FC10A
:1044700082F40401300E82271AEC0BF030C182F472
:104480000401300E82271AEC0BF031C182F40401D2
:10449000300E82271AEC0BF004012E0E826F1AECFC
:1044A0000BF032C182F40401300E82271AEC0BF0BB
:1044B00033C182F40401300E82271AEC0BF00401A0
:1044C0006D0E826F1AEC0BF01200120EF6EC07F074
:1044D000E8CF00F1130EF6EC07F0E8CF01F1140E6F
:1044E000F6EC07F0E8CF02F1150EF6EC07F0E8CF96
:1044F00003F101010A0E046F000E056F000E066F36
:10450000000E076FB0EC28F0000E046F120E056F5E
:10451000000E066F000E076FD0EC28F03DEC29F07E
:104520002AC182F40401300E82271AEC0BF02BC151
:1045300082F40401300E82271AEC0BF02CC182F4B5
:104540000401300E82271AEC0BF02DC182F4040115
:10455000300E82271AEC0BF02EC182F40401300ECB
:1045600082271AEC0BF02FC182F40401300E82274F
:104570001AEC0BF030C182F40401300E82271AECE1
:104580000BF004012E0E826F1AEC0BF031C182F495
:104590000401300E82271AEC0BF032C182F40401C0
:1045A000300E82271AEC0BF033C182F40401300E76
:1045B00082271AEC0BF00401730E826F1AEC0BF0D9
:1045C00012000A0EF6EC07F0E8CF00F10B0EF6EC45
:1045D00007F0E8CF01F10C0EF6EC07F0E8CF02F19E
:1045E0000D0EF6EC07F0E8CF03F116EF23F0060E00
:1045F000F6EC07F0E8CF00F1070EF6EC07F0E8CF95
:1046000001F1080EF6EC07F0E8CF02F1090EF6EC26
:1046100007F0E8CF03F116EF23F001019AEC29F03F
:10462000078457C100F158C101F107940101E80E58
:10463000046F800E056F000E066F000E076FB0EC62
:1046400028F0000E046F040E056F000E066F000EBA
:10465000076FD0EC28F0880E046F130E056F000E64
:10466000066F000E076F9FEC28F00A0E046F000E15
:10467000056F000E066F000E076FD0EC28F03DECC2
:1046800029F0010129674AEF23F00401200E826F0F
:104690004DEF23F004012D0E826F1AEC0BF030C1A8
:1046A00082F40401300E82271AEC0BF031C182F43F
:1046B0000401300E82271AEC0BF032C182F404019F
:1046C000300E82271AEC0BF004012E0E826F1AECCA
:1046D0000BF033C182F40401300E82271AEC0BF088
:1046E0000401430E826F1AEC0BF0120087C32AF10B
:1046F00088C32BF189C32CF18AC32DF18BC32EF112
:104700008CC32FF18DC330F18EC331F190C332F1E0
:1047100091C333F10101296BE8EC29F05FEC29F03A
:104720000101000E046F000E056F010E066F000EF2
:10473000076FB0EC28F00E0E0C6E00C10BF0DFEC32
:1047400007F00F0E0C6E01C10BF0DFEC07F0100E3E
:104750000C6E02C10BF0DFEC07F0110E0C6E03C102
:104760000BF0DFEC07F004017A0E826F1AEC0BF00D
:1047700004012C0E826F1AEC0BF00401350E826FCF
:104780001AEC0BF004012C0E826F1AEC0BF0F2EC19
:1047900021F0FAEF1DF087C32AF188C32BF189C3FA
:1047A0002CF18AC32DF18BC32EF18CC32FF18DC355
:1047B00030F18EC331F190C332F191C333F1010175
:1047C000296BE8EC29F05FEC29F0880E046F130EDA
:1047D000056F000E066F000E076FA4EC28F0000EA8
:1047E000046F040E056F000E066F000E076FB0EC2D
:1047F00028F00101E80E046F800E056F000E066FB1
:10480000000E076FD0EC28F00A0E0C6E00C10BF002
:10481000DFEC07F00B0E0C6E01C10BF0DFEC07F0C4
:104820000C0E0C6E02C10BF0DFEC07F00D0E0C6EDF
:1048300003C10BF0DFEC07F004017A0E826F1AEC73
:104840000BF004012C0E826F1AEC0BF00401360EF3
:10485000826F1AEC0BF004012C0E826F1AEC0BF035
:10486000E1EC22F0FAEF1DF087C32AF188C32BF1A7
:1048700089C32CF18AC32DF18BC32EF18CC32FF188
:104880008DC330F18FC331F190C332F191C333F155
:104890000101E8EC29F05FEC29F0000E046F120E24
:1048A000056F000E066F000E076FB0EC28F00101D7
:1048B0000A0E046F000E056F000E066F000E076FE4
:1048C000D0EC28F0120E0C6E00C10BF0DFEC07F0FC
:1048D000130E0C6E01C10BF0DFEC07F0140E0C6E22
:1048E00002C10BF0DFEC07F0150E0C6E03C10BF0EC
:1048F000DFEC07F004017A0E826F1AEC0BF0040172
:104900002C0E826F1AEC0BF00401370E826F1AEC3A
:104910000BF004012C0E826F1AEC0BF065EC22F008
:10492000FAEF1DF087C32AF188C32BF189C32CF15C
:104930008AC32DF18BC32EF18CC32FF18DC330F1BF
:104940008EC331F190C332F191C333F10101296B70
:10495000E8EC29F05FEC29F0880E046F130E056F68
:10496000000E066F000E076FA4EC28F0000E046F17
:10497000040E056F000E066F000E076FB0EC28F0F6
:104980000101E80E046F800E056F000E066F000E29
:10499000076FD0EC28F0060E0C6E00C10BF0DFECB8
:1049A00007F0070E0C6E01C10BF0DFEC07F0080EEC
:1049B0000C6E02C10BF0DFEC07F0090E0C6E03C1A8
:1049C0000BF0DFEC07F004017A0E826F1AEC0BF0AB
:1049D00004012C0E826F1AEC0BF00401380E826F6A
:1049E0001AEC0BF004012C0E826F1AEC0BF0F7ECB2
:1049F00022F0FAEF1DF081A8B9EF25F007A872EFB9
:104A000025F00101800E006F1A0E016F060E026F75
:104A1000000E036F4BC104F14CC105F14DC106F10D
:104A20004EC107F19FEC28F003BFB9EF25F01AEC57
:104A300027F04BC100F14CC101F14DC102F14EC153
:104A400003F10782ACEC27F018C104F119C105F19C
:104A50001AC106F11BC107F1F80E006FCD0E016FF0
:104A6000660E026F030E036F9FEC28F00E0E0C6EA5
:104A700000C10BF0DFEC07F00F0E0C6E01C10BF064
:104A8000DFEC07F0100E0C6E02C10BF0DFEC07F04C
:104A9000110E0C6E03C10BF0DFEC07F0078401016F
:104AA0009AEC29F057C100F158C101F107940A0EA0
:104AB0000C6E00C10BF0DFEC07F00B0E0C6E01C1A9
:104AC0000BF0DFEC07F00C0E0C6E02C10BF0DFEC0C
:104AD00007F00D0E0C6E03C10BF0DFEC07F007982A
:104AE000B9EF25F007AAB9EF25F0078401019AEC88
:104AF00029F057C100F158C101F10794060E0C6E60
:104B000000C10BF0DFEC07F0070E0C6E01C10BF0DB
:104B1000DFEC07F0080E0C6E02C10BF0DFEC07F0C3
:104B2000090E0C6E03C10BF0DFEC07F0078462C1C5
:104B300000F163C101F164C102F165C103F10794A1
:104B4000120E0C6E00C10BF0DFEC07F0130E0C6EB2
:104B500001C10BF0DFEC07F0140E0C6E02C10BF07C
:104B6000DFEC07F0150E0C6E03C10BF0DFEC07F065
:104B7000079A0401805181197F0B0BE09EA809D090
:104B800014EE00F081517F0BE126E750812B0F01DD
:104B9000AD6E05012F51010A13E081AAE0EF25F067
:104BA00005012F51000A0AE00FB8E0EF25F00501DA
:104BB0003067E0EF25F00FB8E0EF25F0C0EF33F0FD
:104BC00081B8F5EF25F003EC2CF005012F51020A16
:104BD00002E0F5EF25F05C2FF5EF25F05BC55CF505
:104BE0000501010E306F3C0E316F83EF0AF00601B4
:104BF0003251385D3351D8A0010F395D800BD8A4F4
:104C000006EF26F032C638F633C639F61200060132
:104C10003251365D3351D8A0010F375D800BD8B4C7
:104C200016EF26F032C636F633C637F61200078482
:104C30001AC632F61BC633F61CC638F61DC639F640
:104C4000F7EC25F01EC632F61FC633F6F7EC25F05A
:104C500020C632F621C633F6F7EC25F01AC632F636
:104C60001BC633F61CC636F61DC637F607EC26F013
:104C70001EC632F61FC633F607EC26F020C632F603
:104C800021C633F607EC26F03851365F3951D8A0EB
:104C90003929375F9AEC29F036C600F137C601F1A1
:104CA000A6EC29F000C13AF601C13BF622C632F665
:104CB00023C633F624C638F625C639F6F7EC25F0B8
:104CC00026C632F627C633F6F7EC25F028C632F6AC
:104CD00029C633F6F7EC25F022C632F623C633F6A2
:104CE00024C636F625C637F607EC26F026C632F679
:104CF00027C633F607EC26F028C632F629C633F667
:104D000007EC26F03851365F3951D8A03929375F82
:104D10009AEC29F036C600F137C601F1A6EC29F06D
:104D200000C13CF601C13DF62AC632F62BC633F669
:104D30002CC638F62DC639F6F7EC25F02EC632F61D
:104D40002FC633F6F7EC25F030C632F631C633F60F
:104D5000F7EC25F02AC632F62BC633F62CC636F60B
:104D60002DC637F607EC26F02EC632F62FC633F6E0
:104D700007EC26F030C632F631C633F607EC26F0E3
:104D80003851365F3951D8A03929375F9AEC29F06C
:104D900036C600F137C601F1A6EC29F000C13EF697
:104DA00001C13FF63AC632F63BC633F63CC636F68C
:104DB0003DC637F607EC26F03EC632F63FC633F660
:104DC00007EC26F00794120018C100F119C101F197
:104DD0001AC102F11BC103F1000E046F000E056F32
:104DE000010E066F000E076FD0EC28F029A10FEF1F
:104DF00027F02051D8B40FEF27F018C100F119C1E6
:104E000001F11AC102F11BC103F1000E046F000E83
:104E1000056F0A0E066F000E076FD0EC28F0120027
:104E200001010451001305510113065102130751EA
:104E3000031312000101186B196B1A6B1B6B120024
:104E40002AC182F40401300E82271AEC0BF02BC128
:104E500082F40401300E82271AEC0BF02CC182F48C
:104E60000401300E82271AEC0BF02DC182F40401EC
:104E7000300E82271AEC0BF02EC182F40401300EA2
:104E800082271AEC0BF02FC182F40401300E822726
:104E90001AEC0BF030C182F40401300E82271AECB8
:104EA0000BF031C182F40401300E82271AEC0BF0B2
:104EB00032C182F40401300E82271AEC0BF033C1A8
:104EC00082F40401300E82271AEC0BF012002FC17D
:104ED00082F40401300E82271AEC0BF030C182F408
:104EE0000401300E82271AEC0BF031C182F4040168
:104EF000300E82271AEC0BF032C182F40401300E1E
:104F000082271AEC0BF033C182F40401300E8227A1
:104F10001AEC0BF01200060E116E060E126E060E43
:104F2000136E112E91EF27F0122E91EF27F0132E12
:104F300091EF27F08B84020E116E020E126E020E9C
:104F4000136E112EA1EF27F0122EA1EF27F0132ED2
:104F5000A1EF27F08B9412000101005305E10153EA
:104F600003E1025301E1002B6FEC28F09AEC29F0E9
:104F70003951006F3A51016F420E046F4B0E056FAD
:104F8000000E066F000E076FB0EC28F000C104F1B0
:104F900001C105F102C106F103C107F118C100F119
:104FA00019C101F11AC102F11BC103F107B2DDEF12
:104FB00027F0A4EC28F0DFEF27F09FEC28F000C1E9
:104FC00018F101C119F102C11AF103C11BF112005C
:104FD0009AEC29F059C100F15AC101F1060EF6EC24
:104FE00007F0E8CF04F1070EF6EC07F0E8CF05F183
:104FF000080EF6EC07F0E8CF06F1090EF6EC07F024
:10500000E8CF07F19FEC28F000C124F101C125F1A0
:1050100002C126F103C127F1290E046F000E056FAE
:10502000000E066F000E076FB0EC28F0EE0E046F56
:10503000430E056F000E066F000E076FA4EC28F0FC
:1050400024C104F125C105F126C106F127C107F1EC
:10505000B0EC28F000C11CF101C11DF102C11EF12C
:1050600003C11FF1120EF6EC07F0E8CF04F1130EA6
:10507000F6EC07F0E8CF05F1140EF6EC07F0E8CFF8
:1050800006F1150EF6EC07F0E8CF07F10D0E006FF4
:10509000000E016F000E026F000E036FB0EC28F0DF
:1050A000180E046F000E056F000E066F000E076FDE
:1050B000D0EC28F01CC104F11DC105F11EC106F1A0
:1050C0001FC107F1A4EC28F06A0E046F2A0E056FC9
:1050D000000E066F000E076F9FEC28F01200BF0E47
:1050E000FA6E200E3A6F396BD890003701370237CD
:1050F0000337D8B080EF28F03A2F75EF28F0390742
:105100003A070353D8B412000331070B80093F6FED
:1051100003390F0B010F396F80EC5FF0406F3905D9
:1051200080EC5FF0405D405F396B3F33D8B039278A
:1051300039333FA995EF28F040513927120001017A
:10514000BFEC29F0D8B01200010103510719346FE8
:1051500082EC29F0D8900751031934AF800F120068
:105160000101346BA6EC29F0D8A0BCEC29F0D8B032
:10517000120091EC29F09AEC29F01F0E366FD2EC58
:1051800029F00B35D8B082EC29F0D8A00335D8B07F
:105190001200362FBFEF28F034B1A9EC29F012002D
:1051A0000101346B04510511061107110008D8A044
:1051B000A6EC29F0D8A0BCEC29F0D8B01200086BFE
:1051C000096B0A6B0B6BD2EC29F01F0E366FD2EC19
:1051D00029F007510B5DD8A4FAEF28F006510A5DBB
:1051E000D8A4FAEF28F00551095DD8A4FAEF28F009
:1051F0000451085DD8A00DEF29F00451085F055156
:10520000D8A0053D095F0651D8A0063D0A5F0751A9
:10521000D8A0073D0B5FD8900081362FE7EF28F02C
:1052200034B1A9EC29F0346BA6EC29F0D890D6EC77
:1052300029F007510B5DD8A42AEF29F006510A5D29
:10524000D8A42AEF29F00551095DD8A42AEF29F046
:105250000451085DD8A039EF29F0003F39EF29F05B
:10526000013F39EF29F0023F39EF29F0032BD8B481
:10527000120034B1A9EC29F012000101346BA6EC44
:1052800029F0D8B01200DBEC29F0200E366F003781
:1052900001370237033711EE33F00A0E376FE73666
:1052A0000A0EE75CD8B0E76EE552372F4FEF29F0D2
:1052B000362F47EF29F034B12981D890120001012F
:1052C0000A0E346F200E366F11EE29F03451376F0D
:1052D0000A0ED890E652D8B0E726E732372F6AEFA9
:1052E00029F00333023301330033362F64EF29F002
:1052F000E750FF0FD8A00335D8B0120029B1A9ECB0
:1053000029F01200045100270551D8B0053D0127AE
:105310000651D8B0063D02270751D8B0073D0327F4
:1053200012000051086F0151096F02510A6F0351B9
:105330000B6F12000101006B016B026B036B12001B
:105340000101046B056B066B076B12000335D8A0D7
:1053500012000351800B001F011F021F031F003F9B
:10536000B9EF29F0013FB9EF29F0023FB9EF29F079
:10537000032B342B032512000735D8A01200075148
:10538000800B041F051F061F071F043FCFEF29F0E6
:10539000053FCFEF29F0063FCFEF29F0072B342B45
:1053A000072512000037013702370337083709375E
:1053B0000A370B3712000101296B2A6B2B6B2C6B00
:1053C0002D6B2E6B2F6B306B316B326B336B12008E
:1053D00001012A510F0B2A6F2B510F0B2B6F2C51F0
:1053E0000F0B2C6F2D510F0B2D6F2E510F0B2E6F9E
:1053F0002F510F0B2F6F30510F0B306F31510F0B9F
:10540000316F32510F0B326F33510F0B336F12006C
:10541000899C000EC76E200EC66E9E96C69EC50E57
:10542000C96EFF0E9EB602D0E82EFCD79E96C69E91
:10543000000EC96EFF0E9EB602D0E82EFCD7C9CF73
:1054400000F69E96C69E000EC96EFF0E9EB602D056
:10545000E82EFCD7C9CF01F6898C1200000EC76E6A
:10546000200EC66E899C9E96C69EC80EC96EFF0E03
:105470009EB602D0E82EFCD79E96C69E000EC96E40
:10548000FF0E9EB602D0E82EFCD7C9CF02F69E963C
:10549000C69E000EC96EFF0E9EB602D0E82EFCD747
:1054A000C9CF03F6898C899C9E96C69ECA0EC96E8A
:1054B000FF0E9EB602D0E82EFCD79E96C69E000E2A
:1054C000C96EFF0E9EB602D0E82EFCD7C9CF0AF6F1
:1054D0009E96C69E000EC96EFF0E9EB602D0E82EA6
:1054E000FCD7C9CF0BF6898C899C9E96C69ECC0EA4
:1054F000C96EFF0E9EB602D0E82EFCD79E96C69EC1
:10550000000EC96EFF0E9EB602D0E82EFCD7C9CFA2
:1055100012F69E96C69E000EC96EFF0E9EB602D073
:10552000E82EFCD7C9CF13F6898C1200000EC76E87
:10553000200EC66E899C9E96C69EE80EC96EFF0E12
:105540009EB602D0E82EFCD79E96C69E000EC96E6F
:10555000FF0E9EB602D0E82EFCD7C9CF1AF69E9653
:10556000C69E000EC96EFF0E9EB602D0E82EFCD776
:10557000C9CF1BF6898C899C9E96C69EEA0EC96E81
:10558000FF0E9EB602D0E82EFCD79E96C69E000E59
:10559000C96EFF0E9EB602D0E82EFCD7C9CF22F608
:1055A0009E96C69E000EC96EFF0E9EB602D0E82ED5
:1055B000FCD7C9CF23F6898C899C9E96C69EEC0E9B
:1055C000C96EFF0E9EB602D0E82EFCD79E96C69EF0
:1055D000000EC96EFF0E9EB602D0E82EFCD7C9CFD2
:1055E0002AF69E96C69E000EC96EFF0E9EB602D08B
:1055F000E82EFCD7C9CF2BF6898C1200000EC76E9F
:10560000200EC66E899C9E96C69E240EC96EFF0E05
:105610009EB602D0E82EFCD79E96C69EE40EC96EBA
:10562000FF0E9EB602D0E82EFCD7898C899C9E96F0
:10563000C69E200EC96EFF0E9EB602D0E82EFCD785
:105640009E96C69E5F0EC96EFF0E9EB602D0E82ED5
:10565000FCD7898C899C9E96C69E210EC96EFF0E32
:105660009EB602D0E82EFCD79E96C69EC00EC96E8E
:10567000FF0E9EB602D0E82EFCD7898C899C9E96A0
:10568000C69E260EC96EFF0E9EB602D0E82EFCD72F
:105690009E96C69E000EC96EFF0E9EB602D0E82EE4
:1056A000FCD7898C12008984000EC76E220EC66E4C
:1056B0009E96C69E000EC96EFF0E9EB602D0E82EC4
:1056C000FCD79E96C69E000EC96EFF0E9EB602D0F7
:1056D000E82EFCD7C9CFABF59E96C69E000EC96ECC
:1056E000FF0E9EB602D0E82EFCD7C9CFACF59E9631
:1056F000C69E000EC96EFF0E9EB602D0E82EFCD7E5
:10570000C9CFADF59E96C69E000EC96EFF0E9EB621
:1057100002D0E82EFCD7C9CFAEF59E96C69E000EED
:10572000C96EFF0E9EB602D0E82EFCD7C9CFAFF5EA
:105730009E96C69E000EC96EFF0E9EB602D0E82E43
:10574000FCD7C9CFB0F59E96C69E000EC96EFF0E5F
:105750009EB602D0E82EFCD7C9CFB1F5899406ECED
:105760002EF012008984000EC76E220EC66E9E9621
:10577000C69E800EC96EFF0E9EB602D0E82EFCD7E4
:105780009E96C69EABC5C9FFFF0E9EB602D0E82E00
:10579000FCD79E96C69EACC5C9FFFF0E9EB602D032
:1057A000E82EFCD79E96C69EADC5C9FFFF0E9EB6DD
:1057B00002D0E82EFCD79E96C69EAEC5C9FFFF0E4E
:1057C0009EB602D0E82EFCD79E96C69EAFC5C9FFF6
:1057D000FF0E9EB602D0E82EFCD79E96C69EB0C5A0
:1057E000C9FFFF0E9EB602D0E82EFCD79E96C69E3D
:1057F000B1C5C9FFFF0E9EB602D0E82EFCD7899432
:1058000006EC2EF012008984000EC76E220EC66EC2
:105810009E96C69E070EC96EFF0E9EB602D0E82E5B
:10582000FCD79E96C69E000EC96EFF0E9EB602D095
:10583000E82EFCD7C9CFABF59E96C69E000EC96E6A
:10584000FF0E9EB602D0E82EFCD7C9CFACF59E96CF
:10585000C69E000EC96EFF0E9EB602D0E82EFCD783
:10586000C9CFADF59E96C69E000EC96EFF0E9EB6C0
:1058700002D0E82EFCD7C9CFAEF5899406EC2EF005
:105880008984000EC76E220EC66E9E96C69E0F0EAF
:10589000C96EFF0E9EB602D0E82EFCD79E96C69E1D
:1058A000000EC96EFF0E9EB602D0E82EFCD7C9CFFF
:1058B000B3F5899406EC2EF012008984000EC76EB1
:1058C000220EC66E9E96C69E870EC96EFF0E9EB6AF
:1058D00002D0E82EFCD79E96C69EABC5C9FFFF0E30
:1058E0009EB602D0E82EFCD79E96C69EACC5C9FFD8
:1058F000FF0E9EB602D0E82EFCD79E96C69EADC582
:10590000C9FFFF0E9EB602D0E82EFCD79E96C69E1B
:10591000AEC5C9FFFF0E9EB602D0E82EFCD7899413
:1059200006EC2EF089849E96C69E8F0EC96EFF0EE1
:105930009EB602D0E82EFCD79E96C69EB3C5C9FF80
:10594000FF0E9EB602D0E82EFCD7899406EC2EF00E
:1059500012008984000EC76E220EC66E9E96C69EE9
:10596000870EC96EFF0E9EB602D0E82EFCD79E961B
:10597000C69E000EC96EFF0E9EB602D0E82EFCD762
:105980009E96C69E800EC96EFF0E9EB602D0E82E71
:10599000FCD79E96C69E800EC96EFF0E9EB602D0A4
:1059A000E82EFCD79E96C69E800EC96EFF0E9EB650
:1059B00002D0E82EFCD7899406EC2EF089849E96BE
:1059C000C69E8F0EC96EFF0E9EB602D0E82EFCD783
:1059D0009E96C69E010EC96EFF0E9EB602D0E82EA0
:1059E000FCD7899406EC2EF012008984000EC76E55
:1059F000220EC66E9E96C69E870EC96EFF0E9EB67E
:105A000002D0E82EFCD79E96C69E000EC96EFF0EF1
:105A10009EB602D0E82EFCD79E96C69E000EC96E9A
:105A2000FF0E9EB602D0E82EFCD79E96C69E800E34
:105A3000C96EFF0E9EB602D0E82EFCD79E96C69E7B
:105A4000800EC96EFF0E9EB602D0E82EFCD7899458
:105A500006EC2EF089849E96C69E8F0EC96EFF0EB0
:105A60009EB602D0E82EFCD79E96C69E010EC96E49
:105A7000FF0E9EB602D0E82EFCD7899406EC2EF0DD
:105A800012008984000EC76E220EC66E9E96C69EB8
:105A90008F0EC96EFF0E9EB602D0E82EFCD706EC24
:105AA0002EF09E96C69E810EC96EFF0E9EB602D047
:105AB000E82EFCD7899406EC2EF08984000EC76E80
:105AC000220EC66E9E96C69E8F0EC96EFF0E9EB6A5
:105AD00002D0E82EFCD706EC2EF09E96C69E010E54
:105AE000C96EFF0E9EB602D0E82EFCD7899406EC54
:105AF0002EF089849E96C69E910EC96EFF0E9EB6AC
:105B000002D0E82EFCD706EC2EF09E96C69EA50E7F
:105B1000C96EFF0E9EB602D0E82EFCD7899406EC23
:105B20002EF012008984000EC76E220EC66E9E965D
:105B3000C69E8F0EC96EFF0E9EB602D0E82EFCD711
:105B400006EC2EF09E96C69E810EC96EFF0E9EB686
:105B500002D0E82EFCD7899406EC2EF0120089843E
:105B6000000EC76E220EC66E9E96C69E8F0EC96E22
:105B7000FF0E9EB602D0E82EFCD706EC2EF09E96C5
:105B8000C69E010EC96EFF0E9EB602D0E82EFCD74F
:105B9000899406EC2EF012008984000EC76E220E46
:105BA000C66E9E96C69E910EC96EFF0E9EB602D020
:105BB000E82EFCD706EC2EF09E96C69EA50EC96E6A
:105BC000FF0E9EB602D0E82EFCD7899406EC2EF08C
:105BD00012008984000EC76E220EC66E9E96C69E67
:105BE000910EC96EFF0E9EB602D0E82EFCD706ECD1
:105BF0002EF09E96C69E000EC96EFF0E9EB602D077
:105C0000E82EFCD7899406EC2EF01200050EE82E43
:105C1000FED712000501256B266B276B286B899A2E
:105C2000400EC76E200EC66E9E96C69E030EC96EAF
:105C3000FF0E9EB602D0E82EFCD79E96C69E27C5C4
:105C4000C9FFFF0E9EB602D0E82EFCD79E96C69ED8
:105C500026C5C9FFFF0E9EB602D0E82EFCD79E9641
:105C6000C69E25C5C9FFFF0E9EB602D0E82EFCD702
:105C70009E96C69EC952FF0E9EB602D0E82EFCD755
:105C8000898A0F01C950FF0A01E1120005012E5156
:105C9000130A05E005012E51170A0CE01200050158
:105CA000E00E256FFF0E266F0F0E276F000E286F78
:105CB00063EF2EF00501E00E256FFF0E266FFF0E3D
:105CC000276F000E286F899A400EC76E200EC66E91
:105CD0009E96C69E030EC96EFF0E9EB602D0E82E9B
:105CE000FCD79E96C69E27C5C9FFFF0E9EB602D062
:105CF000E82EFCD79E96C69E26C5C9FFFF0E9EB60F
:105D000002D0E82EFCD79E96C69E25C5C9FFFF0E81
:105D10009EB602D0E82EFCD79E96C69EC952FF0EB4
:105D20009EB602D0E82EFCD7898A0F01C950FF0A1F
:105D30001DE005012E51130A05E005012E51170A39
:105D40000BE012000501000E256F000E266F100EED
:105D5000276F000E286F12000501000E256F000E40
:105D6000266F000E276F010E286F12000501256BAC
:105D7000266B276B286B05012E51130A05E00501E0
:105D80002E51170A0CE012000501000E216F000EC3
:105D9000226F040E236F000E246FD8EF2EF0050142
:105DA000000E216F000E226F800E236F000E246FF5
:105DB00021C500F122C501F123C502F124C503F17B
:105DC00025C504F126C505F127C506F128C507F14B
:105DD00010EC27F000C125F501C126F502C127F519
:105DE00003C128F5899A400EC76E200EC66E9E9696
:105DF000C69E030EC96EFF0E9EB602D0E82EFCD7DB
:105E00009E96C69E27C5C9FFFF0E9EB602D0E82EFD
:105E1000FCD79E96C69E26C5C9FFFF0E9EB602D031
:105E2000E82EFCD79E96C69E25C5C9FFFF0E9EB6DE
:105E300002D0E82EFCD79E96C69EC952FF0E9EB693
:105E400002D0E82EFCD7898AC950FF0A08E104C1B4
:105E500025F505C126F506C127F507C128F5D89017
:105E6000050124332333223321332151E00B216FE9
:105E7000216742EF2FF0226742EF2FF0236742EFB6
:105E80002FF02467D8EF2EF00501200E2527E86AB1
:105E90002623E86A2723E86A28231200E86A050116
:105EA0002E51130A06E005012E51170A0BE0020ECF
:105EB000120005012851000A03E12751F00B07E009
:105EC000010E120005012851000A01E0010E120026
:105ED00029C500F12AC501F12BC502F12CC503F13A
:105EE00025C504F126C505F127C506F128C507F12A
:105EF0009FEC28F003BF12004EEC2FF05FE1899A6F
:105F0000400EC76E200EC66E9E96C69E060EC96EC9
:105F1000FF0E9EB602D0E82EFCD7898A899A9E96FB
:105F2000C69E020EC96EFF0E9EB602D0E82EFCD7AA
:105F30009E96C69E27C5C9FFFF0E9EB602D0E82ECC
:105F4000FCD79E96C69E26C5C9FFFF0E9EB602D000
:105F5000E82EFCD79E96C69E25C5C9FFFF0E9EB6AD
:105F600002D0E82EFCD79E96C69E000EC96EFF0E8C
:105F70009EB602D0E82EFCD7898A899A9E96C69E44
:105F8000050EC96EFF0E9EB602D0E82EFCD79E9677
:105F9000C69EC952FF0E9EB602D0E82EFCD7C9B0ED
:105FA000C7EF2FF0898A0501200E2527E86A2623EE
:105FB000E86A2723E86A282368EF2FF01200899AFD
:105FC000400EC76E200EC66E9E96C69E060EC96E09
:105FD000FF0E9EB602D0E82EFCD7898A899A9E963B
:105FE000C69EC70EC96EFF0E9EB602D0E82EFCD725
:105FF000898A0501256B266B276B286B1200899A0D
:10600000400EC76E200EC66E9E96C69E050EC96EC9
:10601000FF0E9EB602D0E82EFCD79E96C69EC952B1
:10602000FF0E9EB602D0E82EFCD7C9CF33F5898A81
:106030001200899A400EC76E200EC66E9E96C69EAE
:10604000B90EC96EFF0E9EB602D0E82EFCD7898A23
:106050001200899A400EC76E200EC66E9E96C69E8E
:10606000AB0EC96EFF0E9EB602D0E82EFCD7898A11
:10607000FF0EE82EFED712004EEC2FF0D8A412002F
:10608000899A400EC76E200EC66E9E96C69E030E5F
:10609000C96EFF0E9EB602D0E82EFCD79E96C69E15
:1060A00027C5C9FFFF0E9EB602D0E82EFCD79E96EC
:1060B000C69E26C5C9FFFF0E9EB602D0E82EFCD7AD
:1060C0009E96C69E25C5C9FFFF0E9EB602D0E82E3D
:1060D000FCD79E96C69EC952FF0E9EB602D0E82EF1
:1060E000FCD7898A0F01C950FF0AD8A433EF33F0D7
:1060F0000501FE0E336F53EC2BF0ABC534F5ACC588
:1061000035F5ADC536F5AEC537F5AFC538F5B0C513
:1061100039F5B1C53AF50784B6C166F1B7C167F183
:10612000B8C168F1B9C169F14BC14FF14CC150F12F
:106130004DC151F14EC152F157C159F158C15AF1F7
:1061400024EC1EF000C13BF501C13CF502C13DF558
:1061500003C13EF505015D67B5EF30F05E67B5EF51
:1061600030F05F67B5EF30F06067B9EF30F0C6EF41
:1061700030F05DC504F15EC505F15FC506F160C58F
:1061800007F19FEC28F003BF33EF33F059C13FF51F
:106190005AC140F5B5C541F5B6C542F517EC26F034
:1061A00036C645F537C646F506014067DFEF30F0E5
:1061B0004167DFEF30F04267DFEF30F04367E3EF36
:1061C00030F0F4EF30F09AEC29F0A0EC29F036C66C
:1061D00000F137C601F140C604F141C605F19FEC5C
:1061E00028F003AF33EF33F00101036B026B1AC6E3
:1061F00000F11BC601F101AF02EF31F0FF0E026F9B
:10620000FF0E036F0101076B066B1CC604F11DC670
:1062100005F105AF10EF31F0FF0E066FFF0E076FAF
:10622000A4EC28F00101076B066B1EC604F11FC623
:1062300005F105AF20EF31F0FF0E066FFF0E076F7F
:10624000A4EC28F00101076B066B20C604F121C6FF
:1062500005F105AF30EF31F0FF0E066FFF0E076F4F
:10626000A4EC28F0D890010103330233013300334A
:10627000D8900101033302330133003300C147F5E5
:1062800001C148F50101036B026B22C600F123C670
:1062900001F101AF50EF31F0FF0E026FFF0E036FFF
:1062A0000101076B066B24C604F125C605F105AF95
:1062B0005EEF31F0FF0E066FFF0E076FA4EC28F0C3
:1062C0000101076B066B26C604F127C605F105AF71
:1062D0006EEF31F0FF0E066FFF0E076FA4EC28F093
:1062E0000101076B066B28C604F129C605F105AF4D
:1062F0007EEF31F0FF0E066FFF0E076FA4EC28F063
:10630000D89001010333023301330033D8900101E7
:10631000033302330133003300C149F501C14AF5AB
:106320000101036B026B2AC600F12BC601F101AF1C
:106330009EEF31F0FF0E026FFF0E036F0101076B3E
:10634000066B2CC604F12DC605F105AFACEF31F09C
:10635000FF0E066FFF0E076FA4EC28F00101076B1C
:10636000066B2EC604F12FC605F105AFBCEF31F068
:10637000FF0E066FFF0E076FA4EC28F00101076BFC
:10638000066B30C604F131C605F105AFCCEF31F034
:10639000FF0E066FFF0E076FA4EC28F0D8900101E6
:1063A0000333023301330033D89001010333023346
:1063B0000133003300C14BF501C14CF50101036B02
:1063C000026B02C600F103C601F101AFECEF31F040
:1063D000FF0E026FFF0E036F0101076B066B04C611
:1063E00004F105C605F105AFFAEF31F0FF0E066FB7
:1063F000FF0E076FA4EC28F00101076B066B06C6C1
:1064000004F107C605F105AF0AEF32F0FF0E066F83
:10641000FF0E076FA4EC28F00101076B066B08C69E
:1064200004F109C605F105AF1AEF32F0FF0E066F51
:10643000FF0E076FA4EC28F0D8900101033302335C
:1064400001330033D89001010333023301330033A9
:1064500000C14DF501C14EF50101036B026B0AC687
:1064600000F10BC601F101AF3AEF32F0FF0E026FFF
:10647000FF0E036F0101076B066B0CC604F10DC61E
:1064800005F105AF48EF32F0FF0E066FFF0E076F04
:10649000A4EC28F00101076B066B0EC604F10FC6D1
:1064A00005F105AF58EF32F0FF0E066FFF0E076FD4
:1064B000A4EC28F00101076B066B10C604F111C6AD
:1064C00005F105AF68EF32F0FF0E066FFF0E076FA4
:1064D000A4EC28F0D89001010333023301330033D8
:1064E000D8900101033302330133003300C14FF56B
:1064F00001C150F50101036B026B12C600F113C616
:1065000001F101AF88EF32F0FF0E026FFF0E036F53
:106510000101076B066B14C604F115C605F105AF42
:1065200096EF32F0FF0E066FFF0E076FA4EC28F017
:106530000101076B066B16C604F117C605F105AF1E
:10654000A6EF32F0FF0E066FFF0E076FA4EC28F0E7
:106550000101076B066B18C604F119C605F105AFFA
:10656000B6EF32F0FF0E066FFF0E076FA4EC28F0B7
:10657000D89001010333023301330033D890010175
:10658000033302330133003300C151F501C152F529
:1065900007940501210E326F899A400EC76E200EB6
:1065A000C66E9E96C69E060EC96EFF0E9EB602D0A1
:1065B000E82EFCD7898A899A9E96C69E020EC96EDD
:1065C000FF0E9EB602D0E82EFCD79E96C69E27C52B
:1065D000C9FFFF0E9EB602D0E82EFCD79E96C69E3F
:1065E00026C5C9FFFF0E9EB602D0E82EFCD79E96A8
:1065F000C69E25C5C9FFFF0E9EB602D0E82EFCD769
:1066000025EE33F0322F02D011EF33F09E96C69E66
:10661000DECFC9FFFF0E9EB602D0E82EFCD702EFF8
:1066200033F0898A899A9E96C69E050EC96EFF0E22
:106630009EB602D0E82EFCD79E96C69EC952FF0E8B
:106640009EB602D0E82EFCD7C9B01CEF33F0898A81
:106650000501200E2527E86A2623E86A2723E86A31
:1066600028238BEC27F0120021C500F122C501F18F
:1066700023C502F124C503F1899A400EC76E200E8E
:10668000C66E9E96C69E0B0EC96EFF0E9EB602D0BB
:10669000E82EFCD79E96C69E02C1C9FFFF0E9EB68D
:1066A00002D0E82EFCD79E96C69E01C1C9FFFF0E00
:1066B0009EB602D0E82EFCD79E96C69E00C1C9FFAA
:1066C000FF0E9EB602D0E82EFCD79E96C69EC952FB
:1066D000FF0E9EB602D0E82EFCD725EE33F0050162
:1066E000200E326F9E96C69EC952FF0E9EB602D0F5
:1066F000E82EFCD7C9CFDEFF322F72EF33F0898A44
:106700001200899A400EC76E200EC66E9E96C69ED7
:10671000900EC96EFF0E9EB602D0E82EFCD79E9654
:10672000C69E000EC96EFF0E9EB602D0E82EFCD7A4
:106730009E96C69E000EC96EFF0E9EB602D0E82E33
:10674000FCD79E96C69E000EC96EFF0E9EB602D066
:10675000E82EFCD79E96C69EC952FF0E9EB602D06A
:10676000E82EFCD7C9CF2DF59E96C69EC952FF0EC6
:106770009EB602D0E82EFCD7C9CF2EF5898A12002A
:106780008BEC27F0B5C5E8FFD70802E38BEC27F0C8
:10679000B5C5E8FFC80802E38BEC27F0B5C5E8FFF4
:1067A000B90802E38BEC27F0B5C5E8FFAA0802E3BD
:1067B0008BEC27F0B5C5E8FF9B0802E38BEC27F0D4
:1067C00003EC2CF019EC30F0F29CF29E8B94C69AFC
:1067D000C290898C9482948C720ED36ED3A4FED70F
:1067E00089968A909390FF0EE8CF00F0E82EFED7AE
:1067F000002EFCD78150F294F29A9E909D909E922A
:106800009D92F298F292F290F286F28E0300FF00CF
:10BF0000E844F926000C160C2B0C3F0C520C640C68
:10BF1000760C860C960CA50CB30CC10CCF0CDC0C6B
:06BF2000E80CF40C000C1B
:00000001FF
